:020000040800F2
:10000000680A00202D020008F16C0008F36C00085B
:10001000F76C0008FB6C0008FF6C00080000000093
:10002000000000000000000000000000036D000858
:10003000056D000800000000076D0008450200087B
:10004000470200084702000847020008470200086C
:10005000470200084702000847020008470200085C
:10006000470200084702000847020008470200084C
:10007000470200084702000847020008470200083C
:10008000470200084702000847020008470200082C
:10009000470200084702000847020008470200081C
:1000A000470200084702000847020008470200080C
:1000B0002D270008470200081527000847020008FE
:1000C00047020008470200084702000847020008EC
:1000D00047020008F920000819310008470200080B
:1000E000076B0008470200084702000847020008A3
:1000F00047020008470200084702000847020008BC
:1001000047020008470200084702000847020008AB
:100110004702000847020008D52D000847020008E2
:10012000470200084702000847020008470200088B
:1001300000F002F800F06AF80AA090E8000C82448F
:100140008344AAF10107DA4501D100F05FF8AFF26C
:10015000090EBAE80F0013F0010F18BFFB1A43F0A5
:1001600001031847F8AA000018AB00000A444FF03A
:10017000000C10F8013B13F0070408BF10F8014B06
:100180001D1108BF10F8015B641E05D010F8016B4B
:10019000641E01F8016BF9D113F0080F1EBF10F8AF
:1001A000014BAD1C0C1B09D16D1E58BF01F801CBD2
:1001B000FAD505E014F8016B01F8016B6D1EF9D555
:1001C0009142D6D37047000000230024002500266A
:1001D000103A28BF78C1FBD8520728BF30C148BFAA
:1001E0000B607047662909F0CC81642906F0FA8516
:1001F000002070471FB507F01FFA040000200021FF
:1002000008F0BAF9E0601FBD10B510BD07F03CFB67
:100210001146FFF7EFFF06F0F9FC07F05AFB03B4B5
:10022000FFF7F2FF03BC01F01BFF00000948804705
:1002300009480047FEE7FEE7FEE7FEE7FEE7FEE7C8
:10024000FEE7FEE7FEE7FEE704480549054A064BE0
:10025000704700004B0300083101000868040020CB
:10026000680A002068060020680600200CB50020FF
:10027000019000906C48006840F480306A49086042
:1002800000BF6948006800F4003000900198401CED
:100290000190009818B90198B0F5A06FF1D16248AB
:1002A000006800F4003010B10120009001E000204F
:1002B00000900098012843D15C48006840F010008D
:1002C0005A4908600846006820F0030008600846A4
:1002D000006840F002000860534840685249486096
:1002E0000846406848600846406840F480604860BE
:1002F0000846406820F47C1048600846406840F496
:10030000E81048600846006840F08070086000BF50
:100310004548006800F000700028F9D04248406865
:1003200020F00300404948600846406840F0020061
:10033000486000BF3C48406800F00C000828F9D134
:100340000CBD10B5FFF792FF10BD10B53648006820
:1003500040F00100344908600846406834490840CC
:100360003149486008460068324908402E49086013
:100370000846006820F4802008600846406820F4A1
:10038000FE0048604FF41F008860FFF7DAFF4FF06F
:1003900000602949086010BD10B50021002000222E
:1003A000214B5B6803F00C0121B1042906D0082918
:1003B00028D107E0214B224C236027E01F4B204C23
:1003C000236023E0184B5B6803F47010164B5B68E6
:1003D00003F48032022303EB904022B9194B4343CC
:1003E000174C23600DE0104B5B6803F4003323B11E
:1003F000144B4343124C236003E0104B4343104C17
:10040000236003E00D4B0E4C236000BF00BF064B82
:100410005B68C3F303130C4CE15C094B1B68CB40D6
:10042000074C236010BD0000001002400020024075
:100430000000FFF8FFFFF6FE08ED00E000127A0072
:100440000000002000093D00040000203149014364
:10045000314A1160704770B5002100230F22C47823
:1004600004B32D4C246804F4E064C4F5E064210A6C
:10047000C1F10403CA40447804FA03F184781440BB
:1004800021430901254C0678A155047804F01F0585
:100490000124AC4005786D11AD0005F1E025C5F8EB
:1004A000004109E0047804F01F050124AC401C4D14
:1004B0000678761145F8264070BD1A4A0A40024374
:1004C000154B1B1F1A60704739B1134A121D126871
:1004D0000243114B1B1D1A6006E00F4A121D1268E1
:1004E00082430D4B1B1D1A607047042808D14FF042
:1004F000E021096941F004014FF0E022116107E0B9
:100500004FF0E021096921F004014FF0E022116170
:10051000704700000000FA050CED00E000E400E088
:1005200080E100E080FFFF1F10B50446CC48844204
:1005300008D10121042000F02DFB0021042000F04F
:1005400029FB46E0C748844208D10121082000F079
:1005500021FB0021082000F01DFB3AE0C248844244
:1005600008D10121102000F015FB0021102000F01F
:1005700011FB2EE0BD48844208D10121202000F06B
:1005800009FB0021202000F005FB22E0B84884424E
:1005900008D10121402000F0FDFA0021402000F0A8
:1005A000F9FA16E0B348844208D10121802000F016
:1005B000F1FA0021802000F0EDFA0AE0AE48844212
:1005C00007D10121801500F0E5FA0021A01500F007
:1005D000E1FA10BD10B50121084600F0DBFA002158
:1005E000012000F0D7FA10BD2DE9F04102460025A8
:1005F0000026002000230024002791F803C00CF0FF
:100600000F0591F803C00CF0100CBCF1000F03D0E3
:1006100091F802C04CEA050591F800C0BCF1000F4A
:1006200031D0146800202BE04FF0010C0CFA00F3DD
:10063000B1F800C00CEA03069E4220D183004FF0BF
:100640000F0C0CFA03F7BC4305FA03FC4CEA040454
:1006500091F803C0BCF1280F06D14FF0010C0CFA41
:1006600000FCC2F814C00AE091F803C0BCF1480FC6
:1006700005D14FF0010C0CFA00FCC2F810C0401C70
:100680000828D1D31460B1F800C0BCF1FF0F34DDED
:10069000546800202EE000F1080C4FF0010808FA21
:1006A0000CF3B1F800C00CEA03069E4221D183008E
:1006B0004FF00F0C0CFA03F7BC4305FA03FC4CEAAD
:1006C000040491F803C0BCF1280F05D100F1080C17
:1006D00008FA0CF8C2F8148091F803C0BCF1480F76
:1006E00007D100F1080C4FF0010808FA0CF8C2F825
:1006F0001080401C0828CED35460BDE8F0814FF62E
:10070000FF710180022181700421C170704702468F
:10071000002093680B400BB1012000E000207047DF
:100720000146886880B2704702460020D3680B40BB
:100730000BB1012000E0002070470146C86880B27C
:10074000704701617047416170470AB1016100E083
:1007500041617047C16070474FF480320A43826143
:100760008161826182698269704702460020434B41
:1007700018684FF68073184040EA021008433F4B58
:10078000186070473E49C8617047F0B50A460023BB
:1007900000240021002500F00046B6F1004F02D1F0
:1007A000364EF16901E0354E7168C0F3034583B2FE
:1007B00000F44016B6F5401F08D121F070612F4EAD
:1007C000766826F070662D4F7E6012E000F4801689
:1007D000B6F5801F06D1032606FA05F4A14341F0C1
:1007E000706106E0460D360103FA06F6B14341F0AA
:1007F000706122B1460D360103FA06F6314300F06E
:100800000046B6F1004F02D11C4EF16101E01B4ED3
:100810007160F0BD30B500228B071C0F0F2303FA67
:1008200004F2164B08338C1053F824309343134CC6
:1008300008348D1044F8253023468C1053F82430AA
:100840008C07240F00FA04F423430C4C08348D1059
:1008500044F8253030BD0A49DC310860704700009B
:1008600000080140000C014000100140001401404C
:1008700000180140001C0140002001400000014020
:1008800000002042DF48006840F00100DD490860B8
:1008900008464068DC490840DA4948600846006874
:1008A000DA490840D74908600846006820F48020EB
:1008B00008600846406820F4FE0048604FF41F00BE
:1008C00088607047CF49096821F48031CD4A1160B2
:1008D0001146096821F480211160B0F5803F03D0F2
:1008E000B0F5802F0ED106E0C649096841F4803189
:1008F000C44A116007E0C349096841F4A021C14A14
:10090000116000E000BF00BF704710B50146002233
:10091000002300204A11012A02D1BA4C236806E0C4
:10092000022A02D1B74C236A01E0B64C636A01F097
:100930001F02012494401C400CB1012000E0002063
:1009400010BD38B5002000900024002500BF3120E4
:10095000FFF7DBFF05460098401C00900098B0F5BB
:10096000A06F01D0002DF2D03120FFF7CEFF08B1EB
:10097000012400E00024204638BD01460020A14AA1
:10098000106820F0F80040EAC10010607047A049EC
:1009900008607047024600209A4B586820F47C108B
:1009A00042EA01031843974B58607047984908661C
:1009B000704701460020934A506820F00300084326
:1009C000506070478F48406800F00C007047014647
:1009D00000208C4A506820F0F000084350607047B7
:1009E00001460020874A506820F4E06008435060C8
:1009F000704701460020834A506820F4605040EA66
:100A0000C1005060704729B17E4A527A02437D4B43
:100A10005A7204E07B4A527A82437A4B5A72704788
:100A20007B49D8310860704701460020754A5068FC
:100A300020F440400843506070470021714A203242
:100A40001170704A82F82010012802D004280AD1BF
:100A500004E001216B4A2032117005E00521694A4A
:100A60002032117000E000BF00BF70476949086084
:100A700070476449096A0143624A116270476549D7
:100A800044390860704730B500210022002400235B
:100A90005C4D6D6805F00C0121B1042905D00829D1
:100AA00023D105E05C4D056022E05B4D05601FE051
:100AB000544D6D6805F47012524D6D6805F4803424
:100AC000022505EB92421CB9544D554305600BE0DD
:100AD0004C4D6D6805F400351DB1504D5543056012
:100AE00002E04D4D5543056002E04B4D056000BFEF
:100AF00000BF444D6D6805F0F0010909484D6B5C7D
:100B00000568DD4045603F4D6D6805F4E061090A08
:100B1000434D6B5C4568DD4085603A4D6D6805F47A
:100B20006051C90A3E4D6B5C4568DD40C560354D7E
:100B30006D6805F44041890B3A4D6B5CC568B5FBA7
:100B4000F3F5056130BD29B12E4A526902432D4BA0
:100B50005A6104E02B4A526982432A4B5A6170471A
:100B600029B1284A92690243264B9A6104E0254A3A
:100B700092698243234B9A61704729B1214AD26915
:100B80000243204BDA6104E01E4AD26982431D4BC6
:100B9000DA61704729B11B4AD2680243194BDA6007
:100BA00004E0184AD2688243164BDA60704729B1D4
:100BB000144A12690243134B1A6104E0114A126984
:100BC0008243104B1A6170471249403908607047E0
:100BD0000F49C86470470B49C87170470948406A9B
:100BE00040F0807007494862704701460020054A7E
:100BF00092680A400AB1012000E0002070470149D4
:100C000088727047001002400000FFF8FFFFF6FEF8
:100C1000000042428004424200127A0000093D0076
:100C2000140000202400002010B50446FE48844231
:100C300008D10121C014FFF7ADFF0021E014FFF738
:100C4000A9FFC4E0B4F1804F08D101210846FFF7A5
:100C5000AEFF00210120FFF7AAFFB8E0F34884426D
:100C600008D101210220FFF7A2FF00210220FFF797
:100C70009EFFACE0EE48844208D101210420FFF73A
:100C800096FF00210420FFF792FFA0E0E94884428C
:100C900008D101210820FFF78AFF00210820FFF773
:100CA00086FF94E0E448844208D101211020FFF738
:100CB0007EFF00211020FFF77AFF88E0DF488442A2
:100CC00008D101212020FFF772FF00212020FFF72B
:100CD0006EFF7CE0DA48844208D101214014FFF71E
:100CE00059FF00216014FFF755FF70E0D54884429A
:100CF00009D10121C804FFF74DFF00214FF4002066
:100D0000FFF748FF63E0D048844209D1012108057C
:100D1000FFF740FF00214FF48010FFF73BFF56E044
:100D2000CA48844209D101214805FFF733FF002159
:100D30004FF40010FFF72EFF49E0C548844208D168
:100D400001214020FFF733FF00214020FFF72FFF54
:100D50003DE0C048844208D101218020FFF727FFF1
:100D600000218020FFF723FF31E0BB48844208D1F7
:100D700001218015FFF71BFF0021A015FFF717FFCA
:100D800025E0B648844209D101210804FFF702FF9B
:100D900000214FF48030FFF7FDFE18E0B048844298
:100DA00009D101214804FFF7F5FE00214FF400307E
:100DB000FFF7F0FE0BE0AB48844208D10121880424
:100DC000FFF7E8FE00214FF48020FFF7E3FE10BD9F
:100DD00000220288944B98420ED0994B98420BD037
:100DE000B0F1804F08D0914B984205D0904B98427B
:100DF00002D0904B984204D14FF68F731A404B8823
:100E00001A438D4B984207D08C4B984204D04FF632
:100E1000FF431A40CB881A4302808B8883850B8856
:100E20000385814B98420BD0854B984208D08B4B61
:100E3000984205D08A4B984202D08A4B984201D101
:100E40000B7A038601238382704770B50024002249
:100E50000023058C4FF6FE7635400584028C83888E
:100E6000048B4FF68F752C40B51E2C400D882C43FB
:100E7000751E2A400D892A434D882A436A4DA8428F
:100E80000BD06F4DA84208D0744DA84205D0744DC8
:100E9000A84202D0734DA84213D14FF6F7752A40ED
:100EA0004D892A434FF6FB752A408D882A434FF619
:100EB000FF652B404FF6FF552B408D892B43CD8985
:100EC0002B4383800483CD888586028470BD70B5F2
:100ED000002400220023058C4FF6EF763540058470
:100EE000028C8388048B48F6FF752C404FF6FF4533
:100EF0002C400D884FF6FF7606EA05252C434FF669
:100F0000DF752A400D8906EA05152A434D8806EA51
:100F100005152A43444DA84202D0494DA8421DD18F
:100F20004FF67F752A404D894FF6FF7606EA051584
:100F30002A434FF6BF752A408D8806EA05152A43D5
:100F40004FF6FF352B404FF2FF752B408D8906EA97
:100F500085052B43CD8906EA85052B4383800483D1
:100F6000CD880587028470BD70B50024002200235F
:100F7000058C4FF6FF6635400584028C8388848B90
:100F80004FF68F752C404FF6FC752C400D882C4386
:100F90004FF6FF552A400D894FF6FF7606EA0525E4
:100FA0002A434D8806EA05252A431F4DA84202D050
:100FB000234DA8421DD14FF2FF752A404D894FF6AF
:100FC000FF7606EA05252A434FF6FF352A408D882D
:100FD00006EA05252A434EF6FF752B404DF6FF75B0
:100FE0002B408D8906EA05152B43CD8906EA0515A8
:100FF0002B4383808483CD888587028470BD70B540
:10100000002200230024058C4EF6FF76354005842F
:10101000038C8488828B48F6FF752A404FF6FF4583
:101020002A400D8820E00000002C01400004004010
:1010300000080040000C0040001000400014004078
:1010400000340140004C0140005001400054014078
:1010500000180040001C00400020004000400140FB
:1010600000440140004801404FF6FF7606EA05259E
:101070002A434DF6FF752B400D8906EA05352B43B3
:101080004D8806EA05352B43FA4DA84202D0FA4DA9
:10109000A84208D14BF6FF752C408D894FF6FF769C
:1010A00006EA85152C4384808283CD88A0F84050C1
:1010B000038470BD828B4FF2FF331A408283828B90
:1010C0004FF6FF7303EA01231A4382837047F0B59A
:1010D0000C461546002200210026078C4EF6FF7CA8
:1010E00007EA0C070784828B018C4FF6FF7707EA2B
:1010F000043640F6FF473A404FF6FF7707EA0527E8
:101100003A434FF6FF7707EA03373A43D94FB842DD
:101110000ED0D94FB8420BD0B0F1804F08D0D74F86
:10112000B84205D0D64FB84202D0D64FB84206D109
:101130004DF6FF77394046F48057394305E047F6CE
:10114000FF57394044F48057394382830184F0BD0E
:10115000828B4FF6F3731A408283828B0A43828319
:101160007047F0B50C461546002200210026078C7A
:101170004FF6FF6C07EA0C070784828B018C4FF651
:10118000FF7707EA04264FF60C773A404FF6FF77D1
:1011900007EA03172F433A43B64FB8420ED0B64F73
:1011A000B8420BD0B0F1804F08D0B44FB84205D050
:1011B000B34FB84202D0B34FB84206D14FF6FF57F3
:1011C000394046F48077394305E04FF2FF57394004
:1011D00044F48077394382830184F0BD028B4FF25F
:1011E000FF331A400283028B4FF6FF7303EA012399
:1011F0001A4302837047F0B50C46154600220021C1
:101200000026078C4FF6EF7C07EA0C070784028B59
:10121000018C4FF6FF7707EA041640F6FF473A4085
:101220004FF6FF7707EA03373A434FF6FF7707EAAF
:1012300005273A438F4FB8420ED08F4FB8420BD09C
:10124000B0F1804F08D08D4FB84205D08C4FB842D6
:1012500002D08C4FB84206D14FF6DF77394046F0C6
:101260001007394305E04FF65F77394044F0100727
:10127000394302830184F0BD028B4FF6F3731A40A9
:101280000283028B0A4302837047F0B50C46154671
:1012900000220021068C4FF6FE773E400684028B2A
:1012A000018C4FF60C7632407E1C06EA03162E4364
:1012B0003243704EB0420ED06F4EB0420BD0B0F100
:1012C000804F08D06D4EB04205D06D4EB04202D076
:1012D0006C4EB04206D14FF6FD76314044F0010627
:1012E000314305E04FF6F576314044F001063143D5
:1012F00002830184F0BD70B505460C465D48854209
:101300000ED05D4885420BD0B5F1804F08D05B48C8
:10131000854205D05A48854202D05A48854200D1BC
:1013200000E000BF208850B92389A2886188284640
:10133000FFF7ABFFE1882846FFF79EFF25E02088F6
:1013400004280AD12389A28861882846FFF753FF21
:10135000E1882846FFF742FF17E0208808280AD1D5
:101360002389A28861882846FFF7FBFEE18828468A
:10137000FFF7EEFE09E02389A28861882846FFF77F
:10138000A6FEE1882846FFF795FE70BD2DE9F041E5
:1013900005460C4600260127608808B9022600E0B1
:1013A0000026A088012801D1022700E0012720881B
:1013B000A0B92389A28861882846FFF766FFE188E3
:1013C0002846FFF759FF23893A4631462846FFF75A
:1013D00012FFE1882846FFF701FF13E02389A28866
:1013E00061882846FFF707FFE1882846FFF7F6FEE9
:1013F00023893A4631462846FFF747FFE1882846C9
:10140000FFF73AFFBDE8F0810A884B881A438B88C2
:101410001A43CB881A430B891A434B891A438B8989
:101420001A43A0F8442070474FF6FF7181800021D5
:101430000180C1804180017270470021018041809C
:101440008180C180018141818181C18170470021FA
:1014500001804180012181800021C180018170478C
:101460000021018041808180C18001814181818191
:1014700070470000002C014000340140000400408F
:1014800000080040000C004021B1028842F0010237
:10149000028004E002884FF6FE731A400280704713
:1014A00031B1B0F8442042F40042A0F8442005E0F5
:1014B000B0F84420C2F30E02A0F8442070471AB1DD
:1014C00083890B43838102E083898B438381704747
:1014D0008182704741EA0203A0F8483070471AB190
:1014E00083890B43838102E083898B438381704727
:1014F00001894FF6F8721140018170470A460021B8
:1015000001894FF68F73194011430181704730B53F
:1015100004460D4629462046FFF7F0FF208940F09B
:101520000700208130BD2DE9F04104460D461646E6
:101530001F46602D06D13B46012231462046FFF76B
:101540005AFE05E03B46012231462046FFF79DFE4C
:1015500029462046FFF7D2FF208940F0070020816E
:10156000BDE8F08130B50C4600210189C9B24FF6C3
:10157000FF7505EA0325154325432943018130BD45
:101580002DE9F04105460E4617469846002443468D
:101590003A4631462846FFF7E5FF2C894FF6F870AA
:1015A000044044F007044FF68F70044044F0700488
:1015B0002C81BDE8F081F0B504460D4616461F4665
:1015C0003B46324629462046FFF7CCFF208940F4AF
:1015D00080402081F0BD0185828270470A4600214B
:1015E00001884FF68F731940114301807047F0B5A1
:1015F0000C4615461E460021002200230189028B5D
:10160000038C4FF6F877394021434FF6FC473A40B8
:1016100040F201173A434FF6DD773B404FF6FF7734
:1016200007EA06172F433B43018102830384F0BD81
:101630000A460021018B4FF68F7319401143018335
:1016400070470A460021018B48F6FF7319404FF698
:10165000FF7303EA02231943018370470A460021FE
:10166000818B4FF68F7319401143818370470A466F
:101670000021818B48F6FF7319404FF6FF7303EA90
:10168000022319438183704721B1028842F080020E
:10169000028004E002884FF67F731A400280704790
:1016A00021B1828842F00402828004E082884FF6F1
:1016B000FB731A408280704721B1828842F0080291
:1016C000828004E082884FF6F7731A408280704768
:1016D00021B1828842F00102828004E082884FF6C4
:1016E000FE731A40828070470A460021018B4FF634
:1016F000F77319401143018370470A460021018B9B
:101700004FF2FF7319404FF6FF7303EA02231943A8
:10171000018370470A460021818B4FF6F773194009
:101720001143818370470A460021818B4FF2FF737A
:1017300019404FF6FF7303EA022319438183704770
:101740000A460021018B4FF6FB73194011430183B8
:1017500070470A460021018B4FF6FF3319404FF6C0
:10176000FF7303EA02231943018370470A460021ED
:10177000818B4FF6FB7319401143818370470A46F2
:101780000021818B4FF6FF3319404FF6FF7303EAB8
:1017900002231943818370470A460021018B4FF6CB
:1017A0007F7319401143018370470A460021018B62
:1017B000C1F30E014FF6FF7303EA022319430183BD
:1017C00070470A460021818B4FF67F731940114301
:1017D000818370470A460021818BC1F30E014FF6C9
:1017E000FF7303EA02231943818370470A460021ED
:1017F000018C4FF6FD7319401143018470470A466E
:101800000021018C4FF6F773194011430184704792
:101810000A460021018C4FF6DF7319404FF6FF7323
:1018200003EA02131943018470470A460021018C20
:101830004FF67F7319404FF6FF7303EA0213194303
:10184000018470470A460021018C4FF6FF5319406E
:101850004FF6FF7303EA02231943018470470A46D7
:101860000021018C4FF2FF7319404FF6FF7303EA1A
:1018700002231943018470470A460021018C4DF66A
:10188000FF7319404FF6FF7303EA023319430184D3
:10189000704730B5002301248C40A3B2048C9C43D4
:1018A0000484048C02FA01F5ADB22C43048430BDEB
:1018B00030B5002304248C40A3B2048C9C430484E0
:1018C000048C02FA01F5ADB22C43048430BD70B52E
:1018D0000346002000241846183001258D40ACB284
:1018E0001D8CA5431D8409B1082909D100EB6100B5
:1018F000056825F0700505600568154305600EE074
:101900000D1FC5F34E052844056825F4E045056024
:1019100005684FF6FF7606EA02263543056070BD7E
:1019200021B1028842F00202028004E002884FF6F0
:10193000FD731A400280704721B1028842F0040210
:10194000028004E002884FF6FB731A400280704761
:1019500021B1828842F08002828004E082884FF6C2
:101960007F731A408280704702884FF6F7731A40DF
:10197000028002880A430280704782884FF68F7384
:101980001A40828082880A438280704702894FF61B
:10199000F8731A40028102890A4302817047028962
:1019A0004FF67F731A40028102890A430281704711
:1019B00081847047818570478186704701877047B1
:1019C00081877047A0F84010704702884FF6FF43A8
:1019D0001A40028002880A43028070470146888EBE
:1019E00070470146088F70470146888F704701464F
:1019F000B1F8400070470146888C70470146088D59
:101A0000704702460020138A0B400BB1012000E012
:101A100000207047CA430282704730B5024600205A
:101A200000230024158A05EA0103958905EA0104CB
:101A300013B10CB1012000E0002030BDCA43028286
:101A40007047000010B50446FB48844209D10121CB
:101A50008803FFF79FF800214FF48040FFF79AF8C2
:101A600032E0F648844209D101214804FFF79FF88B
:101A700000214FF40030FFF79AF825E0F048844247
:101A800009D101218804FFF792F800214FF480204A
:101A9000FFF78DF818E0EB48844209D10121C80412
:101AA000FFF785F800214FF40020FFF780F80BE0E6
:101AB000E548844208D101210805FFF778F80021A4
:101AC0004FF48010FFF773F810BD2DE9F04786B092
:101AD00005460E460024A24600BFA1460027B08955
:101AE00000B100BF2F462C8A4CF6FF700440F088EE
:101AF00004432C82AC894EF6F3100440B08831893F
:101B00000843718908430443AC81AC8A4FF6FF4017
:101B10000440B0890443AC8201A8FEF7B4FFC64874
:101B2000874202D1DDF810A001E0DDF80CA0A88901
:101B300000F4004040B10AEBCA0000EB0A10316823
:101B40004900B0FBF1F807E00AEBCA0000EB0A100D
:101B500031688900B0FBF1F86420B8FBF0F00401B3
:101B60002009642101FB1089A88900F4004040B1DC
:101B7000322000EBC900B0FBF1F000F00700044395
:101B800008E0322000EB09106421B0FBF1F000F016
:101B90000F0004432C8106B0BDE8F0874FF41651C6
:101BA000016000218180C18001810C2141810021DF
:101BB0008181704710B502460020108A4FF2FF0362
:101BC00018400B884C8823438C882343CC882343BC
:101BD0001843108210BD0021018041808180C180A6
:101BE000704721B1828942F40052828104E08289E7
:101BF0004DF6FF731A4082817047F0B5034600240A
:101C000000260025002040F66A17B94200D100BF27
:101C10001846C1F3421401F01F06012707FA06F522
:101C2000012C01D10C3004E0022C01D1103000E075
:101C300014301AB107682F43076002E00768AF430A
:101C40000760F0BD1AB1838A0B43838202E0838A66
:101C50008B4383827047028A4FF6F0731A400282E8
:101C6000028A0A430282704782894FF2FF731A4048
:101C7000828182890A438281704721B1828942F040
:101C80000202828104E082894FF6FD731A4082814C
:101C90007047028A4FF6DF731A400282028A0A43B3
:101CA0000282704721B1028A42F48042028204E03B
:101CB000028A4BF6FF731A4002827047C1F3080292
:101CC0008280704701468888C0F308007047818988
:101CD00041F0010181817047028BD2B20283028BF5
:101CE00042EA012202837047028B02F47F420283A0
:101CF000028B0A430283704721B1828A42F020029C
:101D0000828204E0828A4FF6DF731A408282704733
:101D100021B1828A42F01002828204E0828A4FF668
:101D2000EF731A408282704721B1828A42F0080222
:101D3000828204E0828A4FF6F7731A4082827047EB
:101D400021B1828942F40042828103E08289C2F398
:101D50000E028281704721B1828A42F4006282823F
:101D600004E0828A4FF2FF731A4082827047828AAF
:101D70004FF6FB731A408282828A0A43828270473E
:101D800021B1828A42F00202828204E0828A4FF606
:101D9000FD731A408282704702460020B1F5007F31
:101DA00000D100BF13880B400BB1012000E00020E0
:101DB000704701F40072B2F5007F00D100BFCA4342
:101DC0000280704770B502460024002300250020E1
:101DD00040F66A16B14200D100BFC1F3421501F0CE
:101DE0001F03012606FA03F3012D02D19689334021
:101DF00006E0022D02D1168A334001E0968A334074
:101E00000C12012606FA04F41688344013B10CB102
:101E1000012000E0002070BD10B50022002340F634
:101E20006A14A14200D100BF0A1201249440A3B257
:101E3000DC43048010BD0000003801400044004035
:101E400000480040004C00400050004070B5482061
:101E500000F080F900F0C4F800F08EF84FF4E130A3
:101E600000F0C0F800F0AFFA01F084F9002140F66C
:101E70000F6000F0D1FA00F072FE00F00DFD0222BA
:101E80000021084600F0FFFD03220021102000F091
:101E9000FAFD102320A20021582000F0D7FD0C23CA
:101EA0001FA20221002000F0D1FD0C2320A203215B
:101EB000002000F0CBFD102321A20421002000F01F
:101EC000C5FD0C2322A20621002000F0BFFD0C233B
:101ED00023A20721002000F0B9FD00F05AFB47F2D1
:101EE00030504FF08041888400F0A0FB47F2305022
:101EF0001F4908806421084600F0F0FA00F010FB4A
:101F0000642000F041F94FF4FA752C461948058019
:101F1000001D048070BD00006D2F6D696E00000013
:101F20004C656674203A2020202052504D0000005D
:101F300052696768743A2020202052504D000000FA
:101F4000503A202020493A202020443A20202000E6
:101F50005365745F433A2020202052504D0000000A
:101F60005365745F503A202020206D2F6D696E00FC
:101F7000240800403C04004008B501211020FEF771
:101F8000EFFD4FF40050ADF8000010208DF8030075
:101F900003208DF8020069460F48FEF725FB08BDB7
:101FA00070B504460D480068401C0C490860A0420A
:101FB00010D14FF400510848FEF7A9FBC0F1010011
:101FC000C5B22A464FF400510348FEF7BEFB00207D
:101FD0000249086070BD0000001001402800002088
:101FE0007047000010B586B00446012144F2040099
:101FF000FEF7B6FD4FF40070ADF8140018208DF810
:10200000170003208DF8160005A94D48FEF7ECFADD
:102010004FF48060ADF8140004208DF8170005A976
:102020004748FEF7E1FA01940020ADF80800ADF84A
:102030000A00ADF80C00ADF810000C20ADF80E0051
:1020400001A94048FFF741FD012240F225513D48DA
:10205000FFF7D3FD01213B48FFF7C3FD06B010BDDC
:1020600000BF704770B504460D46E1B23548FFF732
:1020700025FE00BF80213348FFF78EFE0028F9D0EF
:10208000204670BD10B5044600BF20212D48FFF743
:1020900083FE0028F9D02B48FFF714FE10BD70B561
:1020A00004460D4640212748FFF783FE802125483E
:1020B000FFF7B2FE13E021782248FFF7FFFD00BFD3
:1020C00040212048FFF768FE0128F9D140211D4832
:1020D000FFF76FFE80211B48FFF79EFE641C281E41
:1020E000A5F10105E7D170BD0022174B1A60174A10
:1020F0001160174A1060704710B540F22551114821
:10210000FFF760FED8B10F48FFF7DCFDC4B20F48FF
:1021100000680D49096888420CD90D4800680470B0
:102120000B480068401C0A49086007480068401CCA
:102130000549086040F225510248FFF76DFE10BDC9
:102140000008014000380140300000203400002029
:102150002C00002010B504466FF00400FEF7C5F90E
:10216000E11704EB5171C1F3C701234A1170104606
:10217000007800EB4001C1EBC0104FF6FF7101EA9F
:10218000C0001E49088010BD01461C4A12884A43FF
:102190004FF0E0235A6100229A6101221A6100BFC8
:1021A0004FF0E022106900F001021AB100F4803211
:1021B000002AF5D000224FF0E0231A619A6170479F
:1021C00001460D4A12784A434FF0E0235A6100223B
:1021D0009A6101221A6100BF4FF0E022106900F0FD
:1021E00001021AB100F48032002AF5D000224FF02B
:1021F000E0231A619A6170473C0000203E000020F5
:10220000002001E0411CC8B20A28FBDB704710B572
:102210004FF400617F48FEF794FA4FF480617D48E7
:10222000FEF78FFAFFF7ECFF4FF400617948FEF7F5
:102230008AFAFFF7E5FF4FF480617648FEF783FAEC
:10224000FFF7DEFF10BD10B54FF400617148FEF7D7
:102250007AFA4FF480616F48FEF773FAFFF7D0FF08
:102260004FF400616B48FEF76CFA10BD70B5044680
:10227000002528E004F0800028B14FF40061654893
:10228000FEF75FFA04E04FF400616248FEF75BFA84
:10229000FFF7B6FF4FF480615E48FEF752FAFFF792
:1022A000AFFF4FF480615B48FEF74DFA072D04D174
:1022B0004FF400615748FEF744FA6006040EFFF73A
:1022C0009FFF681CC5B2082DD4DB70BD10B54FF45C
:1022D00000615048FEF737FAFFF792FF4FF4806134
:1022E0004C48FEF72EFAFFF78BFF4FF48061494808
:1022F000FEF729FAFFF784FF4FF400614548FEF727
:1023000020FA10BD10B54FF400614248FEF719FAEB
:10231000FFF776FF4FF480613E48FEF712FAFFF7B1
:102320006FFF4FF480613B48FEF70DFAFFF768FF3F
:1023300010BD70B505460024002619E06006040EA5
:102340004FF480613348FEF7FCF9FFF759FF4FF473
:1023500000613048FEF7DBF908B1601CC4B24FF4ED
:1023600080612C48FEF7EFF9FFF74AFF701CC6B2F8
:10237000082EE3DB15B9FFF7C5FF01E0FFF7A6FF65
:10238000204670BD10B54FF400612248FEF7D9F920
:10239000FFF736FF4FF480611E48FEF7D2F9FFF7D2
:1023A0002FFF4FF400611B48FEF7B1F908B101247B
:1023B00000E000244FF480611648FEF7C4F9FFF7EF
:1023C0001FFF204610BD08B501210820FEF7C8FBFD
:1023D0004FF44060ADF8000003208DF80200142097
:1023E0008DF8030069460B48FEF7FEF8FFF72BFF58
:1023F00008BD70B50446FFF7E6FFFFF708FF20466B
:10240000FFF734FFFFF7BEFF0546FFF71CFF284626
:1024100070BD0000000C014030B589B005460C4687
:1024200001210220FEF7A9FB681E80B2ADF808006A
:10243000A0B2ADF804000020ADF80A00ADF8060027
:1024400001A9C048FEF7C4FC0121BE48FFF7E2FA2B
:1024500001221146BB48FFF732F801210820FEF7A0
:102460007FFB0320ADF8100018208DF81300032027
:102470008DF8120004A9B448FEF7B6F86020ADF854
:1024800014000120ADF816000020ADF81A00ADF8D8
:102490001C0005A9AB48FEF767FD0821A948FFF716
:1024A000D1F96020ADF814000120ADF8160000202D
:1024B000ADF81A00ADF81C0005A9A248FEF79FFD73
:1024C0000821A048FFF7D8F901219E48FFF7DCF862
:1024D00001219C48FEF7D8FF09B030BD7FB5054605
:1024E0000C466020ADF800000120ADF80200ADF808
:1024F000065069469348FEF737FD08219148FFF7DB
:10250000A1F9ADF8064069468E48FEF778FD08212E
:102510008C48FFF7B1F901218A48FFF7B5F87FBD74
:102520001FB501211020FEF728FB42F20F70ADF815
:10253000080040F2CF20ADF804000020ADF80A00FA
:10254000ADF806008DF80C0001A98048FEF740FCAC
:1025500001217E48FFF75EFA012211467B48FEF713
:10256000AEFF4FF44070FDF771FF36208DF800008C
:1025700005208DF8010000208DF8020001208DF863
:1025800003006846FDF767FF01217048FEF77CFFF6
:102590001FBD00B587B001210846FEF7EEFA012104
:1025A0000420FEF7DDFA0320ADF8000004208DF8CA
:1025B000030069466648FEF717F804A8FEF734FFE3
:1025C0000020ADF810004EF66020ADF81400002099
:1025D000ADF81600ADF8120004A94FF08040FEF7E8
:1025E000F7FB00231A4603214FF08040FEF7FFFF60
:1025F00001A8FEF72CFF0A20ADF80C0001A9400746
:10260000FEF779FE01218807FFF704FA012211463F
:102610009007FEF754FF00214FF08040FFF7C8F904
:1026200001218807FEF730FF07B000BD00B587B075
:1026300001210420FEF7A1FA01210820FEF790FAFB
:10264000C020ADF8000004208DF8030069463E4824
:10265000FDF7CAFF04A8FEF7E7FE0020ADF8100062
:102660004EF66020ADF814000020ADF81600ADF86D
:10267000120004A93748FEF7ABFB00231A460321DA
:102680003448FEF7B4FF01A8FEF7E1FE0A20ADF8DA
:102690000C0001A92F48FEF72EFE01212D48FFF75F
:1026A000B9F9012211462B48FEF709FF00212948FC
:1026B000FFF77EF901212748FEF7E6FE07B000BDCF
:1026C0000146022904D003290CD004291ED113E0AD
:1026D0004FF08042928C10B247F230524FF080435C
:1026E0009A8415E0174A2432128810B247F2305209
:1026F000144B24331A800BE0164A2432128810B28D
:1027000047F23052134B24331A8001E0002000BFFF
:1027100000BF70470F48103000880E481030008806
:1027200020F001000B491031088070474FF08040C5
:10273000008A4FF08040008A20F001004FF0804175
:102740000882704700040040000C01400010004067
:10275000000801400008004010B50446FFF757FD8F
:102760007820FFF783FDFFF70DFE0020FFF77EFDC9
:10277000FFF708FE2046FFF779FDFFF703FEFFF79E
:1027800062FD10BD10B50446FFF741FD7820FFF74C
:102790006DFDFFF7F7FD4020FFF768FDFFF7F2FD45
:1027A0002046FFF763FDFFF7EDFDFFF74CFD10BD81
:1027B00070B504460D461DB1E0B2FFF7E3FF02E03D
:1027C000E0B2FFF7C9FF70BD70B50646002418E0FF
:1027D00004F1B0000021FFF7EBFF00210846FFF7EE
:1027E000E7FF00211020FFF7E3FF002505E00121AE
:1027F0003046FFF7DDFF681CC5B2802DF7DB601C9B
:10280000C4B2082CE4DB70BD06E041F6650100E0CF
:10281000491E0029FCD1401E0028F6D17047014610
:1028200005E0002001E0421CD0B27B28FBDB0A1E41
:10283000A1F10101F5D1704770B504460D4605F1CF
:10284000B0000021FFF7B4FF102141EA141000216D
:10285000FFF7AEFF04F00F000021FFF7A9FF70BDE6
:1028600010B500218D20FFF7A3FF00211420FFF7F2
:102870009FFF0021AF20FFF79BFF10BD10B5002187
:102880008D20FFF795FF00211020FFF791FF002119
:10289000AE20FFF78DFF10BD70B5002418E004F1E5
:1028A000B0000021FFF784FF00210846FFF780FFFA
:1028B00000211020FFF77CFF002505E0012100200A
:1028C000FFF776FF681CC5B2802DF7DB601CC4B231
:1028D000082CE4DB70BD70B5002418E004F1B000F2
:1028E0000021FFF765FF00210846FFF761FF002187
:1028F0001020FFF75DFF002505E001210846FFF7E6
:1029000057FF681CC5B2802DF7DB601CC4B2082CD1
:10291000E4DB70BD2DE9F04707460E469046994628
:1029200000250024A8F12000C5B27F2F02DD00277A
:10293000B01CC6B2B9F1100F24D131463846FFF7AA
:102940007BFF002408E004EB0511BF4A505C012125
:10295000FFF72EFF601CC4B2082CF4DB701CC1B260
:102960003846FFF769FF002409E004EB0511083140
:10297000B54A505C0121FFF71BFF601CC4B2082C54
:10298000F3DB12E031463846FFF756FF00240AE039
:1029900005EB4501AD4A02EB4101085D0121FFF75E
:1029A00007FF601CC4B2062CF2DBBDE8F08710B54F
:1029B0000246012000E050430B1EA1F10104E1B2E8
:1029C000F9D110BD2DE9FF5F074691461E460E9DC9
:1029D0004FF0000A002435E0301B401EC1B20A202F
:1029E000FFF7E5FFB9FBF0F00A21B0FBF1F201FBC4
:1029F0001208BAF1000F14D1701EA04211DDB8F117
:102A0000000F0CD1AB4605EBDB71491001FB0471E3
:102A1000C8B22B4620220199FFF77CFF10E04FF04F
:102A2000010AAB4605EBDB71491001FB0471C8B22A
:102A300008F13001CAB22B460199FFF76BFF00BFC6
:102A4000601CC4B2B442C7DBBDE8FF9F2DE9F04172
:102A500004460F461546984600260FE0AA5D4346F9
:102A600039462046FFF756FF04F10800C4B2782C1F
:102A700002DD0024B81CC7B2701CC6B2A85D0028D5
:102A8000ECD1BDE8F0812DE9F04180460E461546B7
:102A9000002731464046FFF7CFFE00240AE06C4A8B
:102AA00002EB8511085D0121FFF782FE781CC7B299
:102AB000601CC4B2102CF2DB701CC1B24046FFF7A0
:102AC000BBFE00240CE06900491C614A02EB411185
:102AD000085D0121FFF76CFE781CC7B2601CC4B210
:102AE000102CF0DBBDE8F0812DE9F05F06460F46C3
:102AF00090461C46DDF828A04FF0000BE11704EBD0
:102B00005171C910A4EBC10131B92046E11704EBA2
:102B10005171C1F3C70506E02046E11704EB51717E
:102B2000C910491CCDB23D4615E029463046FFF795
:102B300083FEB1460BE059460BF1010B1AF8010078
:102B40000121FFF735FE09F1010000F0FF09C14541
:102B5000F1DB681CC5B2A542E7DBBDE8F09F10B50C
:102B6000FFF731FC4FF44870FFF70EFB0021AE2059
:102B7000FFF71EFE00210846FFF71AFE0021102075
:102B8000FFF716FE00214020FFF712FE0021B020C3
:102B9000FFF70EFE00218120FFF70AFE0021FF2033
:102BA000FFF706FE0021A120FFF702FE0021A6206C
:102BB000FFF7FEFD0021A820FFF7FAFD00213F20CE
:102BC000FFF7F6FD0021C820FFF7F2FD0021D3201A
:102BD000FFF7EEFD00210846FFF7EAFD0021D520B2
:102BE000FFF7E6FD00218020FFF7E2FD0021D8205D
:102BF000FFF7DEFD00210520FFF7DAFD0021D920D7
:102C0000FFF7D6FD0021F120FFF7D2FD0021DA20E9
:102C1000FFF7CEFD00211220FFF7CAFD0021DB20C7
:102C2000FFF7C6FD00213020FFF7C2FD00218D20F7
:102C3000FFF7BEFD00211420FFF7BAFD0021AF20F1
:102C4000FFF7B6FD10BD00009E98000876960008BC
:102C5000400000202DE9FE4355480468204606F058
:102C6000E7F8064632460B4652A102A804F07EF869
:102C7000102302AA04211846FFF7E8FE4F48056812
:102C8000284606F0D5F8064632460B4649A101A86B
:102C900004F06CF8102301AA04213820FFF7D6FEB7
:102CA0004748D0F80080404606F0C2F80646324653
:102CB0000B4640A1684604F059F810236A460421E7
:102CC0006820FFF7C3FEBDE8FE832DE9FC5F0446E4
:102CD0000D462E1B3B48006806F076FA83463848BE
:102CE0000168584606F0D0FA81463748006806F079
:102CF0006BFA009031480168009806F0C5FA8346E7
:102D0000304606F061FA009029480168009806F004
:102D1000BBFA5946019006F0BFFB8246494606F0D1
:102D2000B3F8804606F014FA07462748006825499C
:102D30000860254806603846BDE8FC9F2DE9FC5F29
:102D400004460D462E1B2148006806F03DFA8346D6
:102D50001B480168584606F097FA81461C480068EF
:102D600006F032FA009015480168009806F08CFAD7
:102D70008346304606F028FA00900D480168009816
:102D800006F082FA5946019006F086FB82464946D3
:102D900006F07AF8804606F0DBF907460C48006832
:102DA0000A4908600A4806603846BDE8FC9F0000F2
:102DB0004002002025312E31660000004402002030
:102DC00048020020500200204C020020580200203F
:102DD000540200202DE9F84F01217D48FEF711FE35
:102DE00000287DD001217A48FEF728FE0520FFF754
:102DF000D7F80220FFF764FCA0F5EA4030387549A7
:102E000008600420FFF75CFCA0F5EA403038724906
:102E10000860084600686F49096800EB010A0AEB80
:102E2000DA7040104FF4167148434FF41C6190FB68
:102E3000F1FB584605F0F0FD8046684A684B05F006
:102E400003FE0646674A684B05F0FEFD044605F0A2
:102E5000A9FB664908600846006805F0E9FF0446DA
:102E600022460B4662A1644803F080FF1023624AA9
:102E700000213020FFF7EAFD56480068002804DAF8
:102E8000544800684042534908605348006800288D
:102E900004DA5148006840424F49086057480068CA
:102EA0004FF41C6148434FF4167190FBF1F4214636
:102EB00048480068FFF709FF514908604F4800681B
:102EC0004FF41C6148434FF4167190FBF1F4214616
:102ED00041480068FFF732FF4A490860484800E06F
:102EE00073E0006810F1030F03DB45480068032816
:102EF00006DD4548006842490968084442490860BF
:102F00004048006810F1030F03DB3E4800680328C7
:102F100006DD3E4800683B49096808443B490860B3
:102F20003948006840F6AC51884203DD40F6B830BD
:102F3000354908603548006840F6AC51884203DDE9
:102F400040F6B8303149086040F2DC502E49086044
:102F50002E4908602C4800882D4908802B4800889D
:102F6000091D0880FFF776FE1A4800684FF41671B5
:102F700048434FF41C6190FBF1F0264908600C2097
:102F8000032300900846022102683820FFF71AFD4B
:102F9000114800684FF4167148434FF41C6190FBD0
:102FA000F1F01D4908600C200323009008461946E3
:102FB00002683820FFF706FD0C20032300900F481D
:102FC000062102683020FFF7FDFCBDE8F88F000005
:102FD000001000405C02002060020020A4703D0A46
:102FE000D7A3B03F6F1283C0CA21094080020020DE
:102FF00025322E32660000008D020020740200206F
:103000006C02002070020020640200206802002090
:103010003C040040780200207C02002010B586B0FD
:10302000044601210420FDF79BFD01214804FDF722
:10303000A4FD0420ADF8140018208DF8170003201B
:103040008DF8160005A94648FDF7CEFA0820ADF820
:10305000140004208DF8170005A94148FDF7C4FAB3
:1030600001940020ADF80800ADF80A00ADF80C009E
:10307000ADF810000C20ADF80E0001A93948FEF79C
:1030800024FD4FF4E060FDF7E1F926208DF8000003
:1030900000208DF801008DF8020001208DF803005A
:1030A0006846FDF7D8F9012240F225512D48FEF778
:1030B000A4FD01212B48FEF794FD06B010BD70B5AC
:1030C00004460D4640212748FEF773FE802125481F
:1030D000FEF7A2FE13E021782248FEF7EFFD00BFC5
:1030E00040212048FEF758FE0128F9D140211D4813
:1030F000FEF75FFE80211B48FEF78EFE641C281E33
:10310000A5F10105E7D170BD0022174B1A60174ADF
:103110001160174A1060704710B540F225511148F0
:10312000FEF750FED8B10F48FEF7CCFDC4B20F48F1
:1031300000680D49096888420CD90D480068047080
:103140000B480068401C0A49086007480068401C9A
:103150000549086040F225510248FEF75DFE10BDAA
:103160000008014000440040980200209C0200201A
:103170009402002008B501210820FDF7F1FC4FF46E
:103180007040ADF8000010208DF8030003208DF88A
:10319000020069463748FDF727FA08BD10B5044616
:1031A0004CB94FF480513348FDF7CBFA4FF400513E
:1031B0003048FDF7C8FA012C07D161032D48FDF70F
:1031C000C0FA21032B48FDF7BEFA022C07D1E10219
:1031D0002848FDF7B8FA21032648FDF7B4FA10BDD8
:1031E00010B504464CB94FF400412248FDF7A9FA46
:1031F0004FF480411F48FDF7A6FA012C07D1A10327
:103200001C48FDF79EFAE1031A48FDF79CFA022CD0
:1032100007D161031748FDF796FAA1031548FDF79A
:1032200092FA10BD10B50020FFF7B8FF0020FFF79D
:10323000D7FF10BD10B50120FFF7B0FF0120FFF749
:10324000CFFF10BD10B50120FFF7A8FF0020FFF74A
:10325000C7FF10BD10B50020FFF7A0FF0120FFF74A
:10326000BFFF10BD10B50220FFF798FF0220FFF747
:10327000B7FF10BD000C014008B501210820FDF783
:103280006FFC4FF44070ADF8000010208DF8030083
:1032900003208DF802006946F748FDF7A5F908BD3F
:1032A00010B5F548001D006820F0F000F249091D36
:1032B00008600846006840F0300008600120EF49CF
:1032C0000860EF48D0F8240108B9002010BD0120A3
:1032D000EA49091F0860FEF773FF0020E849C1F8BA
:1032E000A401E6488038006808B10020EEE701201C
:1032F000FEF766FF0020E149091F08600120E5E7AD
:1033000010B5DD48001D006820F0F000DA49091D05
:1033100008600846006840F0300008600020D74987
:10332000091F0860D649C1F8A4010120FEF748FF33
:103330000120D249091F0860D149C1F8A401FEF754
:103340003FFF10BD10B50024CB48001D006820F0E1
:10335000F000C949091D08600846006840F0800077
:1033600008600120C5490860FEF72AFF0120C44912
:10337000C1F8A001FEF724FF0AE0601CC4B2322CA1
:1033800003DDFFF7BDFF002010BD0120FEF718FF91
:10339000BA48803800680028EFD1B849091F086092
:1033A0000120F1E710B50020B449091F0860B248B8
:1033B000001D006820F0F000AF49091D08600846B4
:1033C000006840F0300008600020AD49C1F8A40159
:1033D0000120FEF7F5FE0120A849091F0860FEF74D
:1033E000EFFE0020A649C1F8A00110BD10B50020D5
:1033F000A249091F0860A048001D006820F0F000E5
:103400009D49091D08600846006840F030000860CA
:1034100001209B49C1F8A401FEF7D2FE0120974983
:10342000091F0860FEF7CCFE00209549C1F8A001F5
:1034300010BD70B504469048001D006820F0F000F3
:103440008D49091D08600846006840F0300008609A
:1034500000208A49091F0860002516E0E009874915
:1034600008606006040E0120FEF7AAFE01208449D0
:10347000C1F8A001FEF7A4FE00208049091F0860E2
:103480000120FEF79DFE681CC5B2082DE6DB70BD6D
:103490002DE9F04105460E4617469846FFF700FF16
:1034A00010B90120BDE8F0816906080EFFF7C1FFE1
:1034B000FFF748FF18B9FFF723FF0120F2E7304676
:1034C000FFF7B7FFFFF73EFF00240BE018F80400FA
:1034D000FFF7AFFFFFF736FF18B9FFF711FF002026
:1034E000E0E7641CBC42F1DBFFF70AFF0020D9E7EC
:1034F00070B5054600246048001D006820F0F0000B
:103500005D49091D08600846006840F080000860B9
:10351000002617E000205949091F08600220FEF725
:103520004FFE01205649C1F8A0016006040E534821
:103530008038006808B1601CC4B20220FEF740FE6B
:10354000701CC6B2082EE5DB15B1FFF72BFF01E0BA
:10355000FFF74CFF204670BD2DE9F04106460F46AF
:1035600014461D46FFF79CFE10B90120BDE8F0810E
:103570007106080EFFF75DFFFFF7E4FE18B9FFF7CD
:10358000BFFE0120F2E73846FFF753FFFFF7DAFEF0
:10359000FFF786FE012101EB4601C8B2FFF749FFA4
:1035A000FFF7D0FE0DE0012C04D10020FFF7A0FFB3
:1035B000287003E00120FFF79BFF28706D1C601E40
:1035C000C4B2002CEFD1FFF79BFE0020CEE770B510
:1035D00005460E460024FFF763FE2846FFF729FF45
:1035E000641CFFF7AFFE3046FFF723FF641CFFF7B4
:1035F000A9FEFFF755FE691CC8B2FFF71AFF641C4D
:10360000FFF7A0FE0020FFF773FF0446FFF778FEE8
:10361000204670BD2DE9F0410746884615461E46F6
:103620000024FFF73DFE3846FFF703FFFFF78AFE51
:103630004046FFF7FEFEFFF785FEFFF731FE791CDF
:10364000C8B2FFF7F6FEFFF77DFE00BF0DE0681E73
:10365000A04204D00120FFF74BFF305503E00020CB
:10366000FFF746FF3055601CC4B2AC42EFDBFFF7FA
:1036700047FE2046BDE8F081000C0140A4812142B4
:10368000008021422DE9F04180460D4616461F4636
:103690000024FFF705FE4046FFF7CBFEFFF752FE82
:1036A0002846FFF7C6FEFFF74DFE00BF06E0385D77
:1036B000FFF7BFFEFFF746FE601CC4B2B442F6DB64
:1036C000FFF71EFE0120BDE8F08170B505460E46ED
:1036D000144631462846FFF77AFF2070012070BD5E
:1036E00037B504460D4602AB012229462046FFF7B6
:1036F000C9FF3EBD2DE9F8430746884614461D46DE
:10370000089E6A4641463846FFF7DFFF28B3601C33
:10371000FF2101FA00F0C4F108012944491EFF22EB
:103720000A41104300F0FF09C5F1080006FA00F055
:10373000C6B2C4F1070006419DF8000000EA090086
:1037400000909DF80000304300909DF80020414615
:103750003846FFF7C5FFBDE8F8830020FBE7F8B562
:1037600006460F4614461D466A4639463046FFF760
:10377000ACFF2DB10120A0409DF80010084305E0EA
:103780000120A0409DF8001021EA0000C0B2009086
:103790009DF8002039463046FFF7A2FFF8BD000033
:1037A000014691F90020002A01DD00201EE091F978
:1037B0000020002A01DA042018E091F90120002AF3
:1037C00001DD012012E091F90120002A01DA052033
:1037D0000CE091F90220002A01DD022006E091F9B7
:1037E0000220002A01DA062000E00720704770B5A9
:1037F00005462846FFF7D4FF0446E81CFFF7D0FF34
:1038000044EAC00084B2A81DFFF7CAFF44EA801052
:1038100084B2204670BD70B588B002A905A801F039
:1038200078FF0446072C3FD101A801F0E7F905987D
:1038300005F0CAFC0646019905F026FD054605F08F
:1038400087FC0590069805F0BFFC0646019905F037
:103850001BFD054605F07CFC0690079805F0B4FCBE
:103860000646019905F010FD054605F071FC07902C
:1038700005A802F05EFA684601F0DDF9BDF8001017
:10388000029848430290BDF8001003984843039003
:10389000BDF8001004984843049002A802F0DCFA36
:1038A000FEA003F057FA00BF08B070BD2DE9F04349
:1038B00004460D46DDE907670021012041E0DFF8FD
:1038C00000C43CF81080A0F1010CDFF8F49329F853
:1038D0001C8009F1160C3CF81090A0F1010CDFF8E7
:1038E000E08308F1160828F81C9008F1160C3CF843
:1038F0001090A0F1010C08F1160828F81C9008F1AE
:10390000160C3CF81090A0F1010C08F1160828F8EC
:103910001C9008F1160C3CF81090A0F1010C08F175
:10392000160828F81C9008F1160C3CF81090A0F12D
:10393000010C08F1160828F81C9000F1010C0CF09D
:10394000FF000A28BBDBDFF878C3ACF81240ACF804
:103950002850ACF83E20ACF85430ACF86A60ACF8B3
:1039600080700021002008E0DFF854C33CF910C04B
:10397000614400F1010C0CF0FF000A28F4DB4FF069
:103980000A0C91FBFCFC0FFA8CFCDFF83483A8F8DE
:1039900014C0002100200AE0DFF824C30CF1160C4B
:1039A0003CF910C0614400F1010C0CF0FF000A2842
:1039B000F2DB4FF00A0C91FBFCFC0FFA8CF8DFF8FD
:1039C00000C3ACF82A80002100200AE0DFF8F0C232
:1039D0000CF12C0C3CF910C0614400F1010C0CF00E
:1039E000FF000A28F2DB4FF00A0C91FBFCFC0FFAF7
:1039F0008CF8DFF8CCC2ACF84080002100200AE04F
:103A0000DFF8BCC20CF1420C3CF910C0614400F17B
:103A1000010C0CF0FF000A28F2DB4FF00A0C91FBBE
:103A2000FCFC0FFA8CF8DFF898C2ACF85680002145
:103A300000200AE0DFF888C20CF1580C3CF910C0F5
:103A4000614400F1010C0CF0FF000A28F2DB4FF09A
:103A50000A0C91FBFCFC0FFA8CF8DFF864C2ACF89E
:103A60006C80002100200AE0DFF854C20CF16E0CDB
:103A70003CF910C0614400F1010C0CF0FF000A2871
:103A8000F2DB4FF00A0C91FBFCFC0FFA8CF8DFF82C
:103A900030C2ACF88280BDE8F08338B50446032319
:103AA00002226B21D0200094FFF724FE38BD38B5E8
:103AB0000446022304221B21D0200094FFF71AFEA3
:103AC00038BD38B50446022304221C21D0200094BE
:103AD000FFF710FE38BD10B50446234606226B21C1
:103AE000D020FFF73CFE10BD10B5764B01227521AA
:103AF000D020FFF78FFD7348007810BD10B5FFF799
:103B0000F3FF682801D1012010BD0020FCE710B5AB
:103B10000446234605226A21D020FFF720FE10BD6F
:103B200010B50446234601223721D020FFF717FEA7
:103B300010BD10B50220FFF7B0FF0320FFF7B7FF5D
:103B40000020FFF7BEFF0020FFF7C5FF0020FFF7B2
:103B5000DEFF0020FFF7E4FF10BD38B50020009025
:103B60006B46012275216820FFF7F6FC9DF80000E6
:103B700068280ED000BF5448006800F4E060534944
:103B80000843001D50490860BFF34F8F00BF00BFBE
:103B9000FEE700F040FDE0B9782000F0A4F97820BD
:103BA00000F088FBC82000F066FC02F027F84848C7
:103BB000FFF71DFE044602F02BF840F2731002F0EE
:103BC00068FCC82002F0DEF9FFF725FE012001F0B5
:103BD0005BFD38BD2DE9F04F8DB00AA83D490BAB18
:103BE00006AACDE900103C493C4802F0B1FD394835
:103BF000008800F4807000287AD0069805F0E4FA76
:103C000004464FF09D4105F0ADF93549086007982D
:103C100005F0DAFA04464FF09D4105F0A3F9314969
:103C20000860089805F0D0FA04464FF09D4105F071
:103C300099F92D490860099805F0C6FA04464FF035
:103C40009D4105F08FF929490860274801684FF028
:103C5000804005F019FB019023480168019805F0A8
:103C600013FB82461F4801684FF0404005F00CFBF3
:103C700001901C480168019805F006FB83465146F7
:103C800005F00AFC81464FF07E5105F0FDF8044630
:103C900005F0CEF8CDE9020111482AE0736574748D
:103CA000696E67206269617320737563636573660B
:103CB000756C6C79202E2E2E2E2E2E0D0A000000F3
:103CC0002E030020200300200CED00E00000FA0588
:103CD000C8020020AC020020A6020020A0020020A2
:103CE000B8020020BC020020C0020020C402002054
:103CF0002FE001684FF0804005F0C6FA8346164871
:103D00000168584605F0C0FA8146144801684FF032
:103D1000804005F0B9FA834611480168584605F01D
:103D2000B3FA8246494605F0AFF8044605F080F83C
:103D30000746DDE9022304F05FFB4FF06632094BD2
:103D4000CDE9040104F080FE054604F02BFC064991
:103D500008600DB0BDE8F08FBC020020C00200205A
:103D6000C402002066A64C40B402002038B50446C8
:103D7000FB4890F82400C0B114B10220009001E08B
:103D800000200090F64A1268D17BF54A52681078FC
:103D90006B460122FFF77CFB10B14FF0FF3038BDBE
:103DA0009DF80010EE48417423E0ED48807A10B988
:103DB0004FF0FF30F3E724B1E948407C08B1002020
:103DC000EDE714B10120009001E000200090E44AEA
:103DD0001268D17BE24A526810786B460122FFF7E5
:103DE00057FB10B14FF0FF30D9E79DF80010DC48C9
:103DF00041740020D3E738B5002419E0D8480068A2
:103E0000C07AA04204D0D6480068407DA04200D1CC
:103E10000CE0D349496808786B4601222146FFF738
:103E20009BFB10B14FF0FF3038BD00BF601CC4B227
:103E3000CB4840680079A042E0DC0020F4E770B590
:103E400004460D46C6480068C07AA04204D0C44863
:103E50000068407DA04202D14FF0FF3070BDC048E5
:103E600040680079A04202DC4FF0FF30F6E7BC4921
:103E7000496808782B4601222146FFF76DFBEDE7E4
:103E800038B50446B64890F82300A04201D100207E
:103E900038BD14B13020009001E000200090B048FF
:103EA000807C20B19DF8000040F002000090AC48FA
:103EB00090F8220020B19DF8000040F080000090B2
:103EC000A74A1268117DA64A526810786B460122F3
:103ED000FFF7DEFA10B14FF0FF30D9E7A04880F8C5
:103EE00023400020D4E738B5044604F0700010B138
:103EF0000120009005E014B10020009001E0402076
:103F00000090974A1268917C954A526810786B46E7
:103F10000122FFF7BDFA20B1002191488172481EAD
:103F200038BD9DF8000020F040018D48017300204D
:103F3000009004F0400020B99DF8000040F004001B
:103F4000009004F0200020B99DF8000040F002002D
:103F5000009004F0100020B99DF8000040F001002E
:103F6000009004F0080020B99DF8000040F03800EF
:103F700000907B4A1268D17C794A526810786B466F
:103F80000122FFF785FA20B1002175488172481E91
:103F9000C6E724B1082C02D00020FFF771FF70485B
:103FA0008472002101753220FEF7EEF80020B7E799
:103FB00038B504466A48807CA04201D1002038BD53
:103FC000002C46D0664A12681179654A526810780A
:103FD0006B460122FFF7C0FA10B14FF0FF30EEE759
:103FE0009DF8000020F0200000905D4A12681179D1
:103FF0005B4A526810786B460122FFF749FA10B10C
:104000004FF0FF30DBE70320FEF7BEF80220009000
:10401000534890F8220020B19DF8000040F0800045
:1040200000904F4890F8230020B19DF8000040F028
:10403000300000904A4A1268117D494A526810784F
:104040006B460122FFF724FA002851D04FF0FF30D1
:10405000B5E7434A12681179414A526810786B46B5
:104060000122FFF779FA10B14FF0FF30A7E73C4883
:10407000807A00F0010028B19DF8000040F0200097
:10408000009004E09DF8000020F020000090344AE9
:1040900012681179324A526810786B460122FFF794
:1040A000F7F910B14FF0FF3089E70320FEF76CF805
:1040B0002B4890F8220010B18020009001E00020F1
:1040C0000090274890F8230020B19DF8000040F0B0
:1040D00030000090224A1268117D214A52681078FF
:1040E0006B460122FFF7D4F910B14FF0FF3066E7BD
:1040F0001B488474002062E708B51948807A10B91B
:104100004FF0FF3008BD00200090154A1268D17BA7
:10411000134A526810786B460122FFF7B9F910B1C3
:104120004FF0FF30EEE70E4A126851790C4A5268A0
:1041300010786B460122FFF7ABF910B14FF0FF305A
:10414000E0E7074A12681179054A526810786B4611
:104150000122FFF79DF928B14FF0FF30D2E70000B0
:10416000D8020020F74890F82400002850D00C20F6
:104170000090F44A12681179F24A526810786B463E
:104180000122FFF785F910B14FF0FF30BAE7C020E8
:104190000090EC48807A00F0010020B19DF800000A
:1041A00040F020000090E74A12681179E54A526811
:1041B00010786B460122FFF76BF910B14FF0FF301A
:1041C000A0E7E048407C10B10220009001E0002010
:1041D0000090DC4A1268D17BDA4A526810786B464C
:1041E0000122FFF755F910B14FF0FF308AE70020A8
:1041F0000090D44A12685179D24A526810786B46BE
:104200000122FFF745F9002852D04FF0FF3079E73F
:1042100004200090CB4A12681179CA4A526810787B
:104220006B460122FFF734F910B14FF0FF3069E718
:10423000C448807C20B9C348807A00F0010010B9DE
:104240004020009001E060200090BE4A1268117981
:10425000BC4A526810786B460122FFF719F910B179
:104260004FF0FF304EE7B748407C10B1012000907E
:1042700001E000200090B34A1268D17BB14A526835
:1042800010786B460122FFF703F910B14FF0FF30B1
:1042900038E7AC4A12685179AA4A52681078A94B9B
:1042A00010330122FFF7F4F810B14FF0FF3029E787
:1042B000002027E770B50446002624F00104A14839
:1042C00090F8240008B1002070BD9E48807A10B993
:1042D0004FF0FF30F8E79B48057C807A20409949F1
:1042E00008740846007CA04202D04FF0FF3600E080
:1042F000002614B99348007D18B10120FFF736FD60
:1043000002E00020FFF732FD3CB1FFF7F5FE20B1DF
:104310008C4805744FF0FF30D6E73046D4E738B507
:1043200004468848807A10B94FF0FF3038BDBC2C65
:1043300002DB0120009015E0622C02DB02200090DD
:1043400010E02A2C02DB032000900BE0142C02DB8F
:104350000420009006E00A2C02DB0520009001E01A
:10436000062000907748C07A9DF80010884201D15D
:104370000020DBE7734A12689178724A526810781D
:104380006B460122FFF784F810B14FF0FF30CDE704
:104390009DF800106B48C1720020C7E738B504468D
:1043A000282C02DD4FF0FF3038BDDCB90020FFF7CC
:1043B00067FD00208DF8000007208DF80100614A9C
:1043C0001268917C5F4A526810786B460222FFF7B0
:1043D0005FF810B14FF0FF30E6E700215948017552
:1043E0000020E1E70120FFF74BFD20208DF80000C1
:1043F000012C06D100208DF801000520FFF78FFF6A
:1044000017E0052C06DC01208DF801000520FFF7E0
:1044100086FF0EE0142C06DC02208DF801000A2035
:10442000FFF77DFF05E003208DF801001420FFF762
:1044300076FF9DF80100072101EB8010C0B28DF8D6
:104440000100404A1268917C3E4A526810786B46DF
:104450000222FFF71DF810B14FF0FF30A4E708214A
:104460003848817200210173012101750020FFF796
:1044700021FF002098E738B504463248807A10B909
:104480004FF0FF3038BD2F4890F8240010B14FF0A6
:10449000FF30F7E72B48007D50B134B1282C04DC05
:1044A000E0B2FFF77BFF0020ECE70020FFF776FF8C
:1044B000042C01DA042404E0B4F57A7F01DD4FF422
:1044C0007A744FF47A7090FBF4F0401EC0B2009002
:1044D0001C4A126851781B4A526810786B460122B8
:1044E000FEF7D6FF10B14FF0FF30CBE79DF800008C
:1044F000401C4FF47A7191FBF0F081B21148C181F8
:104500000146C9894810FFF70AFF0020BAE738B50D
:1045100004460C48807A10B94FF0FF3038BD022CA9
:1045200006D0042C07D0082C08D0102C0FD10BE09B
:10453000002000900EE0082000900BE0102000907A
:1045400008E00000D80200201820009002E04FF0A0
:10455000FF30E3E700BFF948407A9DF80010B0EB68
:10456000E10F01D10020D9E7F44A1268D179F34A6A
:10457000526810786B460122FEF78AFF10B14FF0A7
:10458000FF30CBE79DF80000C110EC4841720020DD
:10459000C4E738B50446E948807A10B94FF0FF30D7
:1045A00038BDFA2C09D0B4F5FA7F09D0B4F57A7F7A
:1045B00009D0B4F5FA6F0CD108E0002000900BE0B0
:1045C0000820009008E01020009005E018200090DE
:1045D00002E04FF0FF30E3E700BFD848007A9DF8D3
:1045E0000010B0EBE10F01D10020D9E7D34A1268E7
:1045F0009179D24A526810786B460122FEF748FF43
:1046000010B14FF0FF30CBE79DF80000C010CB4950
:1046100008720020C4E71CB580208DF80000C74A4E
:104620001268917CC54A526810786B460122FEF7E9
:104630002FFF10B14FF0FF301CBD6420FDF7A4FD2B
:1046400000208DF80000BD4A1268917CBB4A526878
:1046500010786B460122FEF71BFF10B14FF0FF30C0
:10466000EAE7B64A1268917DB44A526810786B4600
:104670000622FEF771FF10B14FF0FF30DCE79DF826
:104680000500C007400F9DF8031001F0010140EA4A
:1046900041009DF8011001F0010140EA010494B1CC
:1046A000012C03D10121A548C17431E0022C03D1B2
:1046B0000021A248C1742BE02146A1A002F04AFBD0
:1046C0004FF0FF30B8E79D4A1268D1789B4A526894
:1046D00010786B460122FEF73FFF10B14FF0FF301C
:1046E000AAE79DF8000000F00F042CB99E4802F0E4
:1046F00031FB4FF0FF309FE7042C06D19BA002F066
:1047000029FB01218D48C17402E000218B48C1744E
:10471000FF218A488172FF2088490872FF2187485B
:104720004172C1724FF6FF71C181FF210174817422
:104730000121017380F82210002180F823104175B7
:1047400001751630016041608160163880F82410D0
:1047500080F82510C1844FF4FA60FFF71AFF10B1FA
:104760004FF0FF3068E70220FFF7D1FE10B14FF0A5
:10477000FF3061E72A20FFF7D2FD10B14FF0FF3084
:104780005AE73220FFF777FE10B14FF0FF3053E7C2
:104790000020FFF78FFD10B14FF0FF304CE70020F5
:1047A000FFF706FC10B14FF0FF3045E70020FFF7A0
:1047B0009AFB002040E770477CB504460D465F48F1
:1047C000807A00F0700010B94FF0FF307CBD5B4A7A
:1047D0001268117B594A526810786B460622FEF720
:1047E000BBFE10B14FF0FF30F0E79DF801009DF8DF
:1047F000001040EA012000B220809DF803009DF8DF
:10480000021040EA012000B260809DF805009DF88A
:10481000041040EA012000B2A08015B12846FFF73D
:10482000CAFF0020D2E77CB504460D464348807A93
:1048300000F0080010B94FF0FF307CBD3F4A12680D
:10484000517B3E4A526810786B460622FEF784FE82
:1048500010B14FF0FF30F0E79DF801009DF8001017
:1048600040EA012000B220809DF803009DF802106C
:1048700040EA012000B260809DF805009DF8041018
:1048800040EA012000B2A08015B12846FFF793FF4F
:104890000020D2E72DE9FE4F05460C462748807AD6
:1048A00018B94FF0FF30BDE8FE8F244A1268917BA3
:1048B000224A5268107802AB0222FEF74DFE10B178
:1048C0004FF0FF30EFE79DF809009DF8081040EA2F
:1048D000012006B214B12046FFF76DFF1749496861
:1048E000C88804F089FC154901904968B1F90800AD
:1048F00004F06AFC8346304604F066FC594600909A
:1049000004F0CAFD8246019904F02CFB81461F4940
:1049100004F0BAFA80464FF08F4104F0B5FC074628
:1049200004F016FC28600020BDE710B588B00446EE
:104930001CB94FF0FF3008B010BD29E0D8020020AC
:10494000556E737570706F7274656420736F6674E2
:10495000776172652070726F64756374207265761A
:104960002025642E0A0000000CAC000848616C662B
:104970002073656E736974697669747920706172E9
:104980007420666F756E642E0D0A000000000C42E4
:10499000206830B9606820B9A06810B9002008B05C
:1049A00010BDFA494968087806AB03221146FEF7A4
:1049B000D3FD10B14FF0FF30F1E79DF8180008214A
:1049C00001EB201000F00F00ADF800009DF8190079
:1049D00001EB201000F00F00ADF802009DF81A0066
:1049E00001EB201000F00F00ADF80400206841003A
:1049F000BDF90000403091FBF0F000B2ADF81000BE
:104A000060684100BDF90200403091FBF0F000B257
:104A1000ADF81200A0684100BDF90400403091FBE0
:104A2000F0F000B2ADF81400D8494968087806AB38
:104A300006221146FEF790FD10B14FF0FF30AEE7B1
:104A40009DF819009DF8181040EA012000B2ADF859
:104A500008009DF81B009DF81A1040EA012000B2E2
:104A6000ADF80A009DF81D009DF81C1040EA0120D9
:104A700000B2ADF80C00BDF81000BDF808100844F5
:104A800000B2ADF81000BDF81200BDF80A100844DD
:104A900000B2ADF81200BDF81400BDF80C100844C7
:104AA00000B2ADF81400BDF81000000A8DF818002F
:104AB000BDF81000C0B28DF81900BDF81200000A50
:104AC0008DF81A00BDF81200C0B28DF81B00BDF8B9
:104AD0001400000A8DF81C00BDF81400C0B28DF857
:104AE0001D00AA494968087806AB06221146FEF760
:104AF000CFFC10B14FF0FF3051E700204FE70146E7
:104B0000A248007A30B1012807D0022809D0032832
:104B10000FD10AE0FA2008800EE04FF4FA70088006
:104B20000AE04FF47A70088006E04FF4FA600880DB
:104B300002E00020088000BF00BF0020704701464F
:104B40009248407A30B1012807D0022808D00328C3
:104B50000CD108E0022008700BE00420087008E087
:104B60000820087005E01020087002E04FF0FF30C8
:104B7000704700BF8548C07C18B108784006000E19
:104B800008700020F4E701468048C07A082817D250
:104B9000DFE800F01704070A0D101318BC20088086
:104BA00013E06220088010E02A2008800DE0142025
:104BB00008800AE00A20088007E00520088004E059
:104BC00000BF00BF0020088000BF00BF002070476A
:104BD00001466E4890F8240010B14FF0FF30704746
:104BE0006A48C08908800020F9E701460020088053
:104BF000401E704701464FF0FF3070470146634842
:104C0000007A30B1012807D0022808D003280CD13F
:104C100008E05F4808600BE05E48086008E05E4816
:104C2000086005E05D48086002E04FF0FF30704723
:104C300000BF0020FBE701465448407A30B101280C
:104C400008D002280AD0032810D10BE04FF480408E
:104C500008800EE041F69C7008800AE04FF4805016
:104C6000088006E04FF40060088002E04FF0FF305B
:104C7000704700BF4548C07C10B1088840100880CC
:104C80000020F5E701464148007C0870002070478D
:104C900001463E48807A10B10120087001E00020F2
:104CA00008700020704738B504463848807A10B93B
:104CB0004FF0FF3038BD354A1268117C334A5268D4
:104CC00010786B460222FEF747FC10B14FF0FF3020
:104CD000F0E79DF801009DF8001040EA012000B2C5
:104CE00020800020E6E72DE9FE4F074688469246E1
:104CF0001D46DDF830B000260024244890F824003A
:104D000010B1601EBDE8FE8F002028701F48807A19
:104D100010B94FF0FF30F5E71C48007C10B94FF098
:104D2000FF30EFE71948007C00F0400008B1B01CEC
:104D3000C6B21648007C00F0200008B1B01CC6B214
:104D40001248007C00F0100008B1B01CC6B20F4839
:104D5000007C00F0080008B1B01DC6B20B4A126812
:104D6000917A0A4A526810786B460222FEF7F4FBE9
:104D700010B14FF0FF30C5E79DF801009DF800101D
:104D800040EA0129B1450BDA0020BBE7D802002038
:104D90000000034300008342333303423333834133
:104DA000FC4840684088B9EB600F17DDF94A12688B
:104DB000517CF84A526810786B460122FEF7CCFB12
:104DC00010B14FF0FF309DE79DF8000000F010009B
:104DD00020B1FFF791F96FF0010093E75046FFF71C
:104DE000EAFCEC4A1268D17AEA4A526810786B46BB
:104DF0003246FEF7B1FB10B14FF0FF3082E799FB6E
:104E0000F6F0401E8BF8000000202870B4422AD033
:104E1000E048007C00F0080028B3601C1DF800008A
:104E20001DF8041040EA012000B2A8F80000E01CC0
:104E30001DF80010A01C1DF8000041EA002000B27F
:104E4000A8F80200601D1DF80010201D1DF80000CC
:104E500041EA002000B2A8F80400287840F00800D9
:104E60002870A01D84B2B44213D0CA48007C00F060
:104E7000400070B1601C1DF800001DF8041040EAED
:104E8000012000B23880287840F040002870A01C33
:104E900084B2B44213D0BF48007C00F0200070B14F
:104EA000601C1DF800001DF8041040EA012000B24B
:104EB0007880287840F020002870A01C84B2B4428A
:104EC00013D0B448007C00F0100070B1601C1DF8D5
:104ED00000001DF8041040EA012000B2B8802878D4
:104EE00040F010002870A01C84B200200AE7F8B53A
:104EF00004460F461646A74890F8240010B94FF014
:104F0000FF30F8BDA348807A10B94FF0FF30F8E7C2
:104F1000A04A1268917A9F4A526810786B46022222
:104F2000FEF71AFB10B14FF0FF30EAE79DF80100E1
:104F30009DF8001040EA0125A54203DA00203070F8
:104F4000401EDEE7934840684088B5EB600F17DDF0
:104F5000904A1268517C8F4A526810786B46012241
:104F6000FEF7FAFA10B14FF0FF30CAE79DF80000E3
:104F700000F0100020B1FFF7BFF86FF00100C0E7AC
:104F8000E2B2844B1B68D97A824B5B6818783B4647
:104F9000FEF7E2FA10B14FF0FF30B2E795FBF4F004
:104FA000401E30700020ACE701467A4880F822109D
:104FB000002070477CB5054676494968087801AB02
:104FC00004220D21FEF7C8FA08B107207CBD9DF828
:104FD0000700C0F301109DF8041001F0E00140EA61
:104FE000E1008DF800009DF80700C0F381009DF8F6
:104FF000051001F0E00140EAE1008DF801009DF8A4
:10500000070000F003009DF8061001F0E00140EAFF
:10501000E1008DF8020000241CE01DF8040018B91E
:10502000002045F8240013E05B4845F8240006E022
:1050300055F82400594904F027F945F824001DF8D3
:105040000400401EC0B20DF804000028F0D100BFDB
:10505000601CC4B2032CE0DB0020B7E72DE9FE4F53
:1050600006460F4600256846FFF7A4FF002442E0ED
:1050700056F8240057F82410A0EB010ABAF1000FEB
:1050800001DB514601E0CAF10001084604F09CF83A
:1050900083464FF08F4103F065FF80465DF82400A2
:1050A000002104F021F816D05DF82410404603F0EA
:1050B00059FF82464FF07E5104F0EEF9814629F007
:1050C000004A3748416A504604F0AAF912D201203A
:1050D000A04005430EE03248C169404604F0A0F804
:1050E00005D32F48016A404604F09AF902D2012004
:1050F000A0400543641C032CBADB2846BDE8FE8FA4
:105100002DE9FC5F06460F460025224949680878CC
:1051100001AB03220D21FEF71FFA10B10720BDE8F5
:10512000FC9F9DF8040000F01F008DF804009DF81E
:10513000050000F01F008DF805009DF8060000F046
:105140001F008DF80600002462E056F8240057F88E
:105150002410A0EB010BBBF1000F01DB594601E06D
:10516000CBF10001084604F02FF84FF08F4100907A
:1051700003F0F8FE814601A8005DC0B30849086845
:1051800004F03AF883465946064803F0EBFE8046A1
:105190000FE00000D80200207B14AE3E1D5A843F71
:1051A000B89E000800B04C45FE49404604F06CF83B
:1051B000804601A8005D401EC0B201A90855002824
:1051C000F2D14146484603F0CDFE83464FF07E5172
:1051D00004F062F982462AF0004BF3488169584690
:1051E00004F01EF913D20120A04005430FE0FFE7B1
:1051F000ED480169484604F013F805D3EA484169CF
:10520000484604F00DF902D20120A0400543641C79
:10521000032C9ADB284682E72DE9F04F87B005463C
:105220000C46914601208DF8100000208DF81100E9
:10523000DE4A1268917CDD4A5268107804AB022283
:10524000FEF726F920B14FF0FF3007B0BDE8F08F30
:10525000C820FCF799FF00208DF81000D34A12688F
:10526000D17BD24A5268107804AB0122FEF710F9C4
:1052700010B14FF0FF30E8E7CC4A12685179CB4AC1
:105280005268107804AB0122FEF702F910B14FF01A
:10529000FF30DAE7C54A1268917CC44A5268107838
:1052A00004AB0122FEF7F4F810B14FF0FF30CCE769
:1052B000BE4A1268D17DBD4A5268107804AB012203
:1052C000FEF7E6F810B14FF0FF30BEE7B74A1268BC
:1052D0001179B64A5268107804AB0122FEF7D8F86B
:1052E00010B14FF0FF30B0E70C208DF81000AF4A3E
:1052F00012681179AD4A5268107804AB0122FEF7AA
:10530000C7F810B14FF0FF309FE70F20FCF73CFFCC
:10531000A648806A407A8DF81000A44A12689178F5
:10532000A24A5268107804AB0122FEF7B1F810B11E
:105330004FF0FF3089E79D48806A007A8DF81000B1
:105340009A4A12685178994A5268107804AB01223F
:10535000FEF79EF810B14FF0FF3076E7B9F1000F7D
:1053600007D09248806A807A40F0E0008DF8100003
:1053700004E08E48806A807A8DF810008B4A1268AB
:1053800091798A4A5268107804AB0122FEF780F8BE
:1053900010B14FF0FF3058E7B9F1000F07D0834844
:1053A000806AC07A40F0E0008DF8100003E07E488B
:1053B000C07A8DF810007D4A1268D1797B4A526814
:1053C000107804AB0122FEF763F810B14FF0FF3004
:1053D0003BE7B9F1000F02D0C820FCF7D5FE402012
:1053E0008DF81000714A12681179704A526810786D
:1053F00004AB0122FEF74CF810B14FF0FF3024E768
:1054000078208DF81000694A12685179674A52680D
:10541000107804AB0122FEF73BF810B14FF0FF30DB
:1054200013E761498889FCF7AFFE00208DF8100072
:105430005E4A126851795D4A5268107804AB0122C5
:10544000FEF726F810B14FF0FF30FEE6574A12681B
:10545000917A564A5268107804AB0222FEF77CF823
:1054600010B14FF0FF30F0E69DF811009DF81010DC
:1054700040EA012B0C209BFBF0F0C6B20020A86094
:1054800068602860A06060602060824665E0474AEE
:105490001268D17A454A5268107804AB0C22FEF7A4
:1054A0005BF810B14FF0FF30CFE69DF811009DF88A
:1054B000101040EA012000B2ADF808009DF813007A
:1054C0009DF8121040EA012000B2ADF80A009DF8E4
:1054D00015009DF8141040EA012000B2ADF80C0050
:1054E000BDF90810206808442060BDF90A10606802
:1054F00008446060BDF90C10A0680844A0609DF8E5
:1055000017009DF8161040EA012000B2ADF8000027
:105510009DF819009DF8181040EA012000B2ADF87E
:1055200002009DF81B009DF81A1040EA012000B20D
:10553000ADF80400BDF90010286808442860BDF9E2
:105540000210686808446860BDF90410A86808443F
:10555000A8600AF1010000F0FF0AB24597DB12488B
:10556000D0F800C02868C117090441EA10410704B7
:1055700062460023384601F0C8FB32460023CDE9DD
:10558000020101F0C2FB28600748D0F800C068683B
:10559000C117090441EA1041070462460023384656
:1055A00006E0000054E3853FB89E0008D8020020C2
:1055B00001F0ABFB32460023CDE9020101F0A5FB6F
:1055C0006860FE48D0F800C0A868C117090441EA25
:1055D0001041070462460023384601F096FB32462C
:1055E0000023CDE9020101F090FBA860F348D0F858
:1055F00004C02168C817000440EA11480F0462463D
:1056000000233846414601F080FB32460023CDE9B5
:10561000020101F07AFB2060E848D0F804C060681D
:10562000C117090441EA10410704624600233846C5
:1056300001F06BFB32460023CDE9020101F065FB6E
:105640006060DE48D0F804C0A068C117090441EAD0
:105650001041070462460023384601F056FB3246EB
:105660000023CDE9020101F050FBA060A0680028F2
:1056700004DDA068A0F58030A06003E0A06800F51C
:105680008030A0600020E0E538B50446CC4890F8B2
:105690002400A04201D1002038BD24B3C84890F8AE
:1056A000250010B94FF0FF30F6E70020FEF75EFB53
:1056B0000020FEF77DFCC249C88CFEF7DCFE00200E
:1056C0000090BF49496808786B4601222321FDF705
:1056D000DFFE0121BA4880F824100120FEF746FBC6
:1056E000FEF70AFD13E00020FEF740FBB448007C03
:1056F0000090B349496808786B4601222321FDF7E1
:10570000C7FE0021AE4880F82410FEF7F5FC00200B
:10571000C2E72DE9F04F8DB083460F4602200C9072
:10572000A74890F8240020B10020FFF7ADFF012624
:1057300000E0002603A8FFF7E2F905A8FFF7FFF94C
:1057400001A8FFF720FA02A8FFF742FA9C4890F858
:105750000AA004A8FFF796FA002407E000223946C1
:105760005846FFF759FD00B902E0641C022CF5DB36
:1057700000BF022C01D1002528E0002407E001220F
:1057800006A909A8FFF748FD00B902E0641C022C35
:10579000F5DB00BF022C01D1002517E006A9384631
:1057A000FFF75CFC00F0FF0809A95846FFF7A8FCCA
:1057B00000F0FF090025B9F1000F01D145F0010506
:1057C000B8F1000F01D145F0020500BFFF207C4970
:1057D0000872FF217A484172C1724FF6FF71C18190
:1057E000FF218172017401210173BDF80C00FEF7E5
:1057F000D0FE9DF81400FEF78AFEBDF80400FEF707
:105800008EFDBDF80800FEF736FE5046FEF76BFB36
:105810009DF81000FEF74EFD16B10120FFF734FF92
:1058200028460DB0BDE8F08FF8B504460D46164683
:1058300016B94FF0FF30F8BD6148807A10B94FF0CB
:10584000FF30F8E720128DF80000E0B28DF801007B
:105850009DF8010028445A4949684989884202DD77
:105860004FF0FF30E7E7564A1268117E544A5268FB
:1058700010786B460222FDF70BFE10B14FF0FF309F
:10588000D9E7EAB24E4B1B68597D4D4B5B681878DF
:105890003346FDF7FDFD10B14FF0FF30CBE70020A0
:1058A000C9E7F8B504460D46164616B94FF0FF3065
:1058B000F8BD4348807A10B94FF0FF30F8E7201266
:1058C0008DF80000E0B28DF801009DF80100284439
:1058D0003B4949684989884202DD4FF0FF30E7E7DC
:1058E000374A1268117E364A526810786B46022297
:1058F000FDF7CEFD10B14FF0FF30D9E7EAB2304BE3
:105900001B68597D2E4B5B6818783346FDF724FEE3
:1059100010B14FF0FF30CBE70020C9E72DE9F0438D
:1059200085B005460E4690469946254890F82500D4
:1059300020B14FF0FF3005B0BDE8F08316B94FF04D
:10594000FF30F8E7002423E0281B102801DD102099
:1059500000E0281B87B2321939462046FFF764FF62
:1059600010B14FF0FF30E6E701AA39462046FFF7B5
:1059700098FF10B14FF0FF30DDE730193A4601A92A
:1059800001F0F3FA10B16FF00100D4E7E01984B22E
:10599000AC42D9DB4FEA28208DF8000008F0FF0068
:1059A0008DF80100064A1268917E054A5268107807
:1059B0006B460222FDF76CFD38B103E0B89E00088B
:1059C000D80200204FF0FF30B5E701218A4880F867
:1059D0002510A0F826900020ADE70146864890F8F3
:1059E000240008700020704702464FF0FF307047D7
:1059F00001464FF0FF307047F8B505460F46144694
:105A0000002C70D0B5F5FF5F01DDFF2605E0202DED
:105A100001DA012601E0C5F3471607B90127282C52
:105A200002DD4FF0FF30F8BD7348407D28BB72485F
:105A300090F8240038B10020FFF726FE01216E48BF
:105A400080F8201003E000216B4880F820106A489D
:105A50001630FFF754F868481830FFF770F86648BA
:105A60001A30FFF790F864481C30FFF7B1F862482D
:105A7000817A81771F30FFF705F90020FEF776F96C
:105A80000020FEF78BFC00208DF800005A4A1268B7
:105A90009178594A526810786B460122FDF7F8FC5C
:105AA00010B14FF0FF30BEE740208DF80000524AA1
:105AB0001268D17B504A526810786B460122FDF77C
:105AC000E7FC00B165E08DF800608DF801704A4A8E
:105AD0001268117A484A526810786B460222FDF724
:105AE000D7FC08B155E047E00520FCF74DFB4248E4
:105AF000407A072101EBC000C0B28DF800003E4A99
:105B00001268D1793C4A526810786B460122FDF741
:105B1000BFFC00B13DE020208DF80000012C03D136
:105B200000208DF801000EE0052C03DC01208DF82B
:105B3000010008E0142C03DC02208DF8010002E0D3
:105B400003208DF801009DF80100072101EB801072
:105B5000C0B28DF80100284A1268917C264A52682A
:105B600010786B460222FDF793FC00B111E0012191
:105B700021484175002056E71F4A1632002103E0F4
:105B8000505C00B105E0491C0C29F9D34FF0FF30FF
:105B900049E7FF2018490872FF2117484172C17276
:105BA0004FF6FF71C181FF218172017401210173E0
:105BB0000146887FFEF797F90F49C88AFEF7E9FC8E
:105BC0000D49087EFEF7A3FC0B49488BFEF7A7FBA7
:105BD0000949888BFEF74FFC0749C87FFEF76AFB2F
:105BE000054890F8200010B10120FFF74DFD00217D
:105BF00001484175002016E7D802002010B5C823DF
:105C00004FF48062F74940F6F630FFF787FE10BD8B
:105C100010B586B00446F4A000680390F3A00068B5
:105C20000290F3A000680190F2A00068009004F0D8
:105C3000030003A9085C8DF8140003A8C4F3C10194
:105C4000405C8DF8150003A8C4F38111405C8DF809
:105C5000160004F0030002A9085C8DF8100002A8E9
:105C6000C4F3C101405C8DF8110002A8C4F3811196
:105C7000405C8DF8120005AA032140F22640FFF790
:105C8000D3FD18B14FF0FF3006B010BD04AA0321B8
:105C900040F22A40FFF7C8FD10B14FF0FF30F3E7A4
:105CA000019805900098049004F0040058B19DF804
:105CB000140040F001008DF814009DF8100040F031
:105CC00001008DF8100004F0200058B19DF8150077
:105CD00040F001008DF815009DF8110040F0010022
:105CE0008DF8110004F4807058B19DF8160040F052
:105CF00001008DF816009DF8120040F001008DF8AB
:105D0000120005AA03214FF48860FFF78DFD10B142
:105D10004FF0FF30B8E704AA032140F23140FFF70B
:105D200083FD10B14FF0FF30AEE7B348048100208F
:105D3000AAE71FB50446B048007A00F0030054F803
:105D400020000190AC48007A00F0040010B10198E6
:105D500040420190A848007AC0F3C10054F82000E6
:105D60000290A548007A00F0200010B1029840424D
:105D70000290A148007AC0F3811054F820000390EB
:105D80009D48008900F4807010B103984042039050
:105D90009A49019880FB0101800F40EA810001903F
:105DA0009649029880FB0110820042EA91700290AD
:105DB0009249039880FB0110820042EA917003909F
:105DC0000198000E8DF800000198000C8DF801007C
:105DD0000198000A8DF802000198C0B28DF8030006
:105DE0006A4604214FF47470FFF71EFD18B14FF09E
:105DF000FF3004B010BD0298000E8DF8000002982C
:105E0000000C8DF801000298000A8DF8020002983B
:105E1000C0B28DF803006A4604214FF47570FFF795
:105E200003FD10B14FF0FF30E3E70398000E8DF84B
:105E300000000398000C8DF801000398000A8DF80B
:105E400002000398C0B28DF803006A4604214FF4A3
:105E50007670FFF7E9FCCCE770B588B0064601A87C
:105E6000FEF7E9FEBDF804000021C90341EA5045F0
:105E7000C4036148007A00F0030056F82000059042
:105E80005D48007A00F0040010B10598404205908A
:105E90005948007AC0F3C10056F8200006905648D1
:105EA000007A00F0200010B1069840420690524857
:105EB000007AC0F3811056F8200007904E48008900
:105EC00000F4807010B10798404207900598C11700
:105ED000A0FB042301FB043100FB0510810041EA13
:105EE000927005900698C117A0FB042301FB0431B2
:105EF00000FB0510810041EA927006900798C117D7
:105F0000A0FB042301FB043100FB0510810041EAE2
:105F1000927007900598000E8DF808000598000C07
:105F20008DF809000598000A8DF80A000598C0B29E
:105F30008DF80B000698000E8DF80C000698000CEA
:105F40008DF80D000698000A8DF80E000698C0B274
:105F50008DF80F000798000E8DF810000798000CC0
:105F60008DF811000798000A8DF812000798C0B24A
:105F70008DF8130002AA0C214FF42570FFF754FC92
:105F800008B070BD30B585B004461DA207CA02AB8B
:105F900007C3C82C03DD4FF0FF3005B030BDC8206B
:105FA00090FBF4F0401E85B2280A8DF80000E8B29C
:105FB0008DF801006A46022140F21620FFF734FCFA
:105FC00010B14FF0FF30E8E702AA0C2140F6C120E3
:105FD000FFF72AFC10B14FF0FF30DEE7064884815E
:105FE0000020DAE7E09E00084CCD6C000CC92C00C4
:105FF0003656760026466600B403002009E3CA023E
:10600000FEF2ABC4AAF1DFDFBBAFDFDF0146FC4825
:1060100080890880002070472DE9FC4706460F461E
:1060200006F0070010B1B7F5C86F03DD4FF0FF3081
:10603000BDE8FC87384603F0DFF88146F14902F0FD
:1060400091FF80466846FEF77AFD9DF80000022821
:1060500006D0042816D0082826D0102848D135E0CC
:106060004FF08D41404603F00FF9814603F08CF864
:1060700084B2E549404603F007F9814603F084F80D
:1060800085B238E04FF08C41404603F0FDF8814680
:1060900003F07AF884B2DD49404603F0F5F8814612
:1060A00003F072F885B226E04FF08B41404603F0D2
:1060B000EBF8814603F068F884B2D549404603F016
:1060C000E3F8814603F060F885B214E04FF08A41AE
:1060D000404603F0D9F8814603F056F884B2CD4922
:1060E000404603F0D1F8814603F04EF885B202E055
:1060F0004FF0FF309CE700BF20128DF80400E0B2A3
:106100008DF8050028128DF80600E8B28DF807001A
:1061100006F00100A0B101AA02214FF4EA70FFF7D6
:1061200083FB10B14FF0FF3082E70DF10602022130
:106130004FF49270FFF778FB10B14FF0FF3077E724
:1061400006F00200A0B101AA02214FF4EC70FFF7A3
:106150006BFB10B14FF0FF306AE70DF10602022130
:106160004FF49470FFF760FB10B14FF0FF305FE722
:1061700006F00400A0B101AA02214FF4EE70FFF76F
:1061800053FB10B14FF0FF3052E70DF10602022130
:106190004FF49670FFF748FB10B14FF0FF3047E720
:1061A000002045E738B504460020009004F00100C7
:1061B00020B19DF8000040F03000009004F0020093
:1061C00020B19DF8000040F00C00009004F00400A5
:1061D00020B19DF8000040F0030000906A460121C4
:1061E0004FF4A470FFF720FB38BD38B50446012CEE
:1061F00001DA012402E0042C00DD0424601EC0B298
:1062000000906A46012140F24F10FFF70DFB38BDA8
:1062100038B50446052094FBF0F085B228128DF8BD
:106220000000E8B28DF801006A4602214FF4EF70D9
:10623000FFF7FAFA38BD38B50446052094FBF0F0B4
:1062400085B228128DF80000E8B28DF801006A4688
:1062500002214FF4ED70FFF7E7FA38BDF8B50546B7
:106260000E464FF47A7095FBF0F000FB06F4200E1A
:106270008DF80000200C8DF80100200A8DF8020036
:10628000E0B28DF803006A4604214FF4AE70FFF7C8
:10629000CBFAF8BD38B50446052094FBF0F084B283
:1062A00020128DF80000E0B28DF801006A4602214C
:1062B0004FF4AD70FFF7B8FA38BD38B50446052085
:1062C00094FBF0F084B220128DF80000E0B28DF85B
:1062D00001006A4602214FF4AC70FFF7A5FA38BD01
:1062E00038B5044614B94FF0FF3038BD6A46042172
:1062F0004FF45870FFF7D5FA10B14FF0FF30F4E7C4
:106300009DF8000000069DF8011040EA01409DF84C
:10631000021040EA01209DF803100843206000208D
:10632000E3E738B50446200E8DF80000200C8DF808
:106330000100200A8DF80200E0B28DF803006A46E1
:1063400004214FF45870FFF76FFA38BD38B5044692
:1063500014B94FF0FF3038BD6A4604214FF4717014
:10636000FFF79FFA10B14FF0FF30F4E79DF80000FF
:1063700000069DF8011040EA01409DF8021040EA35
:1063800001209DF80310084300EB8000800020608E
:106390000020E0E738B504461420B4FBF0F4200EEA
:1063A0008DF80000200C8DF80100200A8DF8020005
:1063B000E0B28DF803006A4604214FF47170FFF7D4
:1063C00033FA38BD38B5044664B120208DF800009A
:1063D00028208DF8010030208DF8020038208DF83B
:1063E000030004E0A3220421684600F0EAFD6A46A7
:1063F000042140F69E20FFF717FAFDF77DFE38BD19
:10640000B403002000004843000040460000C0459F
:10641000000040450000C04438B5044664B1C020C7
:106420008DF80000C2208DF80100C4208DF8020014
:10643000C6208DF8030004E08B220421684600F09A
:10644000C0FD6A46042140F69820FFF7EDF9FDF7FC
:1064500053FE38BD3EB504466CB1FDA1D1E9002024
:106460008968CDE9002002916A4609214FF49760BE
:10647000FFF7DAF93EBDF9A2D2E900109268CDE942
:10648000010200916A4609214FF49760FFF7CCF9A9
:10649000F0E73EB5044602208DF80000CA208DF8D2
:1064A0000100E3208DF8020009208DF803006A4600
:1064B00004216820FFF7B8F9A3208DF8000004F04C
:1064C000400048B1C0208DF80100C8208DF80200BE
:1064D000C2208DF8030006E0A3208DF801008DF89E
:1064E00002008DF8030004F4C07048B1C4208DF898
:1064F0000400CC208DF80500C6208DF8060006E0CB
:10650000A3208DF804008DF805008DF80600A32067
:106510008DF807008DF808008DF809006A460A21F9
:1065200040F6A720FFF780F904F0030018B12020FF
:106530008DF8000002E0D8208DF800006A460121A5
:1065400040F6B620FFF770F904F0200018B10120E2
:10655000FFF780FF02E00020FFF77CFF04F4C0702B
:1065600008B304F4807060B1B2208DF800008B2075
:106570008DF80100B6208DF802009B208DF80300F5
:106580000BE0B0208DF8000080208DF80100B420D1
:106590008DF8020090208DF803006A46042140F631
:1065A000A220FFF741F904F0010020B3F8208DF894
:1065B00000006A4601214FF40B60FFF735F9FA211C
:1065C0000720FFF729FD0720FFF7ECFD0120FFF76B
:1065D0000CFE6420FFF71CFE4FF4FA70FFF72BFE51
:1065E000C821A148FFF73AFE2820FFF753FE0A20F2
:1065F000FFF763FE08E0D8208DF800006A4601210D
:106600004FF40B60FFF710F904F0020018B1D92025
:106610008DF8000002E0D8208DF800006A460121C4
:1066200040F23D70FFF700F904F0040018B10120BA
:10663000FFF7F2FE02E00020FFF7EEFE04F010008C
:1066400018B10120FFF7BEFE02E00020FFF7BAFEFE
:1066500044F0080085494881FDF74EFD002083493C
:10666000887304F0400018B10846807B801D887351
:1066700004F4C07020B17D48807B801D7B49887305
:1066800004F0140020B17948807B1030774988737A
:1066900004F0030020B17548807B001D73498873A6
:1066A00000203EBD014671484089088000207047A7
:1066B0002DE9F0410446E07800F0C006E07800F0F3
:1066C0003F05607800F0010098B1EF102846E91707
:1066D00005EB5171C910A5EBC101491C01F0FF0880
:1066E0006248006820B161484146026838469047D8
:1066F00000BF607800F0080030B15C48406818B115
:10670000B0115A4A516888470020BDE8F08110B5A1
:1067100086B0044656A207CA03AB07C357A207CAEE
:106720008DE80700012C09D0022C0ED103AA0B2101
:1067300040F68220FFF778F806B010BD6A460B21BC
:1067400040F68220FFF770F8F6E74FF0FF30F3E7EE
:106750002DE9F04F8DB00746884615469946DDE98C
:10676000166B0024002030804049887B5A4605A9DA
:10677000FEF7BDFB18B1601E0DB0BDE8F08F3B48C1
:10678000807A00F01400002861D09DF81400000603
:106790009DF8151040EA01409DF8161040EA0120CE
:1067A0009DF81710084328609DF8180000069DF812
:1067B000191040EA01409DF81A1040EA01209DF8A6
:1067C0001B10084368609DF81C0000069DF81D1012
:1067D00040EA01409DF81E1040EA01209DF81F107C
:1067E0000843A8609DF8200000069DF8211040EAAB
:1067F00001409DF8221040EA01209DF82310084333
:10680000E86004F11000C4B22868001401906868C0
:1068100000140290A86800140390E8680014049023
:1068200001984043029901FB0100039901FB01001B
:10683000049901FB010ABAF1706F02DBBAF1885FBB
:1068400022DDFDF759FC00203080401E94E721E056
:10685000B8AAB38DB4980D355D000000B8AAAAAAF5
:10686000B088C3C5C700000009E3CA02B403002012
:10687000D8B1B9F38BA391B609B4D900DAB1B9F3A1
:106880008BA391B6DAB4DA00B6F9000040F4807058
:10689000308000BF3448807A00F0400020B305A962
:1068A000601C085C095D40EA012000B2A8F8000005
:1068B00005A9E01C095C05AAA01C105C41EA0020A7
:1068C00000B2A8F8020005A9601D095C201D105C3B
:1068D00041EA002000B2A8F80400A01DC4B2B6F935
:1068E000000040F0080030801F48408900F4C0706C
:1068F00008B305A9601C085C095D40EA012000B2EC
:10690000388005A9E01C095C05AAA01C105C41EABE
:10691000002000B2788005A9601D095C201D105C74
:1069200041EA002000B2B880A01DC4B2B6F9000050
:1069300040F0700030800C48807A00F0030018B1FD
:1069400005A90819FFF7B4FE4846FDF734FF0020FB
:1069500012E70146044801600020704701460248E2
:106960004160002070470000B4030020704770B5FC
:1069700005468D49284602F053FC08D38B4928462A
:1069800002F04EFD03D38A480078012801D101248A
:1069900000E00024204670BD03461846884200DD12
:1069A0000846904200DA104670472DE9FF5F044622
:1069B0008946804803908048029004EB09014842D0
:1069C00002F002FC7D4908607D48006802F030FA60
:1069D00007467C4A7C4B02F037F8054601F0E2FDA1
:1069E000774908607548006802F022FA754A774BCB
:1069F000CDE9000102F028F805460E46704800680F
:106A000002F016FA07462A46334601F0FDFD82469B
:106A100001F0C8FD6A490860084601686C480068D2
:106A200002F032FA6A4908606A496948006802F06F
:106A3000F7FC02D267486649086067496448006805
:106A400002F0EEFB02D26448614908606048029996
:106A5000006802F019FC07465948006880F00046BB
:106A60003046039902F010FC0546394602F014FD49
:106A70005A4908605A480068FFF779FF012803D097
:106A80004B480078012802D1002051490860534842
:106A9000006802F05DFB04B0BDE8F09F2DE9FE4FF9
:106AA00004460D464F4E504F0021204602F0E9FCAF
:106AB00002902946002002F0EFFC0190394601982F
:106AC00002F0E2FB86F0004B00905846029902F07B
:106AD000DBFB8246009902F0DFFC814602F038FBC6
:106AE00080464046BDE8FE8F10B5FDF773F83F487D
:106AF00000683B4908603E49B1F9000002F064FBC0
:106B00003C49086010BD2DE9F0414FF480503A49EE
:106B100008603A48007808B9012000E000203749B1
:106B20000870FFF7E1FF35480078012802D1002006
:106B3000BDE8F0812F48016829480068FFF7AEFFE3
:106B400004462F4801682F480068FFF72EFF0546CE
:106B5000671966192C4A51423846FFF71DFF074650
:106B6000294A51423046FFF717FF06461C48006885
:106B7000FFF7FDFE18B931463846FFF7F7FE002053
:106B8000D6E7012807D10A49097809B9012100E0AF
:106B90000021074A117070470146002901DA484276
:106BA00000E0084670470000000020C200002042BC
:106BB0000C03002000002043CDCC4C3F14030020E8
:106BC000180300209A9999999999E93F9999C93F91
:106BD0001C03002000401C4600401CC6100300207F
:106BE0000403002000006143713D8A3FB40200208D
:106BF000A002002008030020140401400D0300201F
:106C0000600200205C0200200CE5FFFFFBF71EF98C
:106C10004FF41650FCF702FAFCF724FB64E0142052
:106C2000FBF7B2FA06213148FCF76EFA06212F482D
:106C3000FCF745FA2D48C078B12806D12B480079D9
:106C4000B52802D100202949C8702848C078B32847
:106C500006D126480079B72802D100202349C87000
:106C60002248C078B22805D120480079B62801D141
:106C7000FCF7D8FA1D48C078B4280ED11B4800791B
:106C8000B8280AD1FCF7DEFA4FF4FA70FBF77CFA69
:106C9000FCF7C8FA00201549C8701448C078B52818
:106CA00005D112480079B92801D1FCF7DBFA0F4869
:106CB000C078B6280ED10D480079BA280AD1FCF761
:106CC000C9FA4FF4FA70FBF75FFAFCF7ABFA002051
:106CD0000649C8700548C078B82805D1034800792E
:106CE000BC2801D1FCF7A6FA99E70000C4030020F4
:106CF000704700BFFEE700BFFEE700BFFEE700BF32
:106D0000FEE7704770477047704710B54C1084EA33
:106D1000530404D54042C1F1000138BF491E1B4253
:106D200004D55242C3F1000338BF5B1E00F055F991
:106D300014F0804F04D04042C1F1000138BF491E19
:106D400014F0004F04D05242C3F1000338BF5B1E61
:106D500010BD00000FB4044910B503AA029800F05A
:106D600037FC10BC5DF814FB380000200FB41CB5D4
:106D7000074B06AA7B4469460090059800F00FFC7B
:106D80000020694600F01EFC1CBC5DF814FB0000EE
:106D90004D08000070B5044685690068C10601D53C
:106DA000302600E02026C00707D070BDD4E90121BD
:106DB00030469047206A401C20626D1EF6D570BD9B
:106DC00070B5044685690078C00707D170BDD4E965
:106DD000012120209047206A401C20626D1EF6D5BC
:106DE00070BD00002DE9F0410646002410687529A9
:106DF000314616A510D0AFF30080002802DA4042D9
:106E000013A507E031688A0701D512A502E04907FA
:106E100004D511A5012401E0AFF3008000210A226E
:106E200006F1240709E0B0FBF2FCB0FBF2F302FB31
:106E30001C00303078541846491C0028F3D12346F2
:106E40002A463046BDE8F04100F03EB9000000009F
:106E50002D0000002B000000200000002DE9F0476D
:106E60004FF0000A89460446C0F820A02046E16899
:106E70008847002876D0252806D0D4E901219047FC
:106E8000206A401C2062F1E7E1682046002588471F
:106E9000C4F81CA006460027C4F818A02A2E09D062
:106EA000304601F091F938B304EB8708303EC8F85A
:106EB000186019E059F8041B204604EB8702916121
:106EC000E1688847012F064618D1E069002820DADA
:106ED00025F020051DE0D8F8180000EB800006EB37
:106EE00040003038C8F818002046E1688847064658
:106EF00001F06AF90028EED1012F0AD02E2E08D118
:106F00002046E16888477F1C0646022F45F0200591
:106F1000C4DBA069002803DA404245F00105A06106
:106F2000E80701D025F01005B6B1A6F141001928F7
:106F300002D8203645F400654A4631462046256091
:106F40004D46F9F74FF958B1012806D0ED1D25F04F
:106F5000070000F1080989E704E005F1040985E765
:106F600030468AE7206ABDE8F08740EA010310B5A1
:106F70009B070FD1042A0DD310C808C9121F9C42C9
:106F8000F8D020BA19BA884201D9012010BD4FF0BB
:106F9000FF3010BD1AB1D30703D0521C07E0002008
:106FA00010BD10F8013B11F8014B1B1B07D110F865
:106FB000013B11F8014B1B1B01D1921EF1D1184668
:106FC00010BD02F0FF0343EA032242EA024200F04E
:106FD00013BB704770477047704753EA020C00F0CC
:106FE00069802DE9F04B4FF00006002B1FBFB3FA6C
:106FF00083F503FA05F424FA05F65E4012BF164342
:10700000B2FA82F502FA05F4C5F120051EBF22FA94
:1070100005FC44EA0C04203556EA044C4FEA1444BB
:1070200018BF641C4FF000084FF00009904271EB4C
:10703000030C39D3002919BFB1FA81F701FA07F619
:10704000B0FA80F700FA07F6C7F120071EBF20FA52
:1070500007FC46EA0C062037B6FBF4FCA7EB050755
:10706000103F07F01F0BCBF120060CFA0BFB2CFA9C
:1070700006F644BFB3460026202FA4BF5E464FF05D
:10708000000B5BEA060C08BF4FF0010B19EB0B0974
:10709000ABFB027C48EB0608C01B06FB02CC0BFBDB
:1070A00003CC71EB0C01C1E70B4602464146484652
:1070B000BDE8F08B13B54FF000004FF00001AFF3C7
:1070C0000080BDE81C4070472DE9F0470D46994609
:1070D0009246044600F124080168880604D5E06958
:1070E00021F01001216000E00120A84201DD471BD2
:1070F00000E00027A1697A1902EB0900081AA061D3
:107100002078C00602D42046FFF744FE002608E09F
:10711000D4E901211AF806009047206A401C761C29
:1071200020624E45F4DB2078C0060AD52046FFF7E2
:1071300031FE06E0D4E9012130209047206A401C4E
:107140002062381EA7F10107F4DC07E0D4E9012131
:1071500018F805009047206A401C2062281EA5F1FF
:107160000105F3DC2046FFF72BFE2078000602D550
:107170000220BDE8F0870120FBE770472DE9FF4FB3
:107180000C461E464FF0FF378BB0D2E90001DDF808
:1071900060800A908A46C1F30A5505B93D46002130
:1071A00008464FF00000BAF1000F00F4400005DA85
:1071B00000EB80004FF4400101EA50004FEA905983
:1071C000B9F1010F00DDB9460A9850EA4A000ED025
:1071D00044F61050A5F2FF3545432F14B8F1000FC7
:1071E0001ED07542291E1EDDC9F100021CE0B8F157
:1071F000010F4FF0000001D0302103E0F24305E021
:107200002154401CB042FBDB3046002200212154B7
:107210000B99C1F80880C1E900200FB0BDE8F08FDC
:10722000BD1B6D1CDEE74A4600DA694206A800F085
:107230008DFA06AB93E8070003AB83E807005046DE
:107240000A9900F08FFB8DE80700A0F500501F3869
:1072500000900398002D09DD42F21F014A460844C0
:1072600003A90390684600F0EEFD08E0A0F5005089
:107270004A461F3803A90390684600F0F8FD8DE8E0
:1072800007000004000C03D04FF0FF30410800E07D
:107290001046B8F1000F03D00022009215461EE000
:1072A000751E05D400F0CCF9303262556D1EF9D54B
:1072B000B3460122084302D000227F1C04E020785C
:1072C000302801D100227F1E002A099786D01DE0B8
:1072D000112D07DA00F0B4F9303262556D1C50EA16
:1072E0000102F5D1084302D00098C8B10EE0002198
:1072F000681E05E0235C625C63542254401E491CF6
:107300008142F7DBAB46A81B401E0990002004F821
:107310000B000B98099AC0F80880C0E9002B7CE7A5
:1073200011264FF0000859E72DE9F04F8846044632
:10733000D21D22F0070191B0D1E90001CDE90A0187
:1073400000F0CBFE02460B98C00F01D02D2007E0C5
:107350002068810701D52B2002E0202101EAC0002E
:10736000032A099001D0072A05DB0346414620463F
:1073700000F0ACF90BE12078800601D5E06900E06F
:107380000620B8F1650F814606D0B8F1660F18D017
:10739000B8F1670F70D131E00020B9F1110F009002
:1073A00001DB112301E009F101030AAA01A90CA8DC
:1073B000FFF7E4FEDDE90C70002609F101058346C4
:1073C00047E001204B4600904FF000470AAA01A970
:1073D0000CA8FFF7D3FEDDE90DB00C995D46002641
:1073E00010B909F101000D18B9EB050003D4C0F183
:1073F000FF3609F10105A5EB09002BE0B9F1010FFA
:1074000001DA4FF001090020B9F1110F0090484650
:1074100001DD112300E003460AAA01A90CA8FFF729
:10742000ADFEDDE90C704D4600268346207800074E
:107430000AD4AB4500DA5D4601A8012D04DD4119EF
:1074400011F8011C302907D04F4502DA17F1040F5B
:1074500004DA012082460FE06D1EEEE7002F02DC09
:10746000ED1B3E4403E0781CA84200DD7D1CB81BE8
:1074700000F1010A4FF000472078000703D4AA4525
:1074800001DB4FF0FF3A0021B7F1004F0DF1430847
:107490008DF8431024D002202B23002F01DA7F42E5
:1074A0002D230A21021EA0F1010000DC5FB197FB31
:1074B000F1FC97FBF1F201FB1C7C17460CF1300C40
:1074C00008F801CDEEE7A8F1010003702188090555
:1074D00001D5452100E06521A0F1010800F8011C5B
:1074E00009980FA9A1EB0807FF1D00B10120411960
:1074F00001EBEA70A1693844081A401EA0612078A7
:10750000C00602D42046FFF745FC099828B1D4E90B
:1075100001219047206A401C20622078C00622D5B5
:107520002046FFF737FC1EE0002E04DBB34502DDEA
:1075300001A8805D00E03020D4E901219047206A55
:10754000401C2062761CAAF101005FEA000A0AD101
:1075500000F072F8C0680168405CD4E901219047EE
:10756000206A401C2062281EA5F10105DCDC07E032
:10757000D4E9012118F8010B9047206A401C2062D1
:10758000381EA7F10107F3DC2046FFF719FC0320A2
:1075900011B043E601694A1C02610878704700B5E2
:1075A0008FB0CDE901310021059105497944CDE93C
:1075B000031011466846FFF751FC0FB000BD0000F4
:1075C000E5FFFFFF0A6802F8010B0A607047000040
:1075D000074B70B50D467B44FFF7E1FF0446284694
:1075E00000F022F910B14FF0FF3070BD204670BDA1
:1075F0008BAAFFFF4FF000020429C0F0128010F0A8
:10760000030C00F01781CCF1040CBCF1020F18BF81
:1076100000F8012BA8BF20F8022BA1EB0C0100F011
:1076200009B95FEAC17C24BF00F8012B00F8012BE7
:1076300048BF00F8012B7047004870472404002021
:1076400030B5B0F10A024FEA900E71F100034EEA34
:10765000817EB0EB0E0061EB91014FEA101E4EEA05
:10766000017E10EB0E0041EB11114FEA102E4EEA95
:10767000016E10EB0E0041EB11214FEA104E4EEA65
:10768000014E10EB0E0041EB1141401841F1000199
:107690004FEAD00040EA41704FEAD10110EB80057B
:1076A0004FEA810444EA907444EB01046D1944EB01
:1076B0000404521BA3414FF0000348BF0A3200D517
:1076C00030BD401C41F1000130BD00002DE9F0410A
:1076D0001F46044603260168072A01F4006004DB04
:1076E00008B116A505E016A503E008B115A500E050
:1076F00015A521F010002060A069C01EA0610FB187
:10770000401EA0612046FFF745FB4FB1D4E901219F
:1077100038469047206A401C2062C01C206206E068
:10772000206AFAE7D4E9012115F8010B9047761E8B
:10773000F8D22046FFF744FBBDE8F0814E414E00F1
:107740006E616E00494E4600696E66002DE9F04795
:10775000814616468AB0334878440DC88DE80D003E
:1077600030487844801C03AC0DC884E80D0041F615
:107770009B300844372190FBF1F290FBF1F5A5F125
:10778000800501FB12041B3C02D56442012000E08D
:107790000020DFF890A080460027FA44AAF1BE0A34
:1077A0000DE0E00709D03246684607EB47010AEBD7
:1077B000810100F05CFB8DE8070064107F1C002C49
:1077C000EFD1184F7F44AC3F18E0E80714D007EB27
:1077D00004100DF1180A90E80E008AE80E00C06847
:1077E000F04201D198190890324606A903A800F08A
:1077F0003EFB03AB83E807006D10641C002DE4D151
:1078000032466946B8F1000F03A802D000F01BFB16
:1078100001E000F02CFBC9E90001C9F808200AB01A
:10782000BDE8F08798340000007B00F080007047CE
:107830004FF0000200B5134694469646203922BF09
:10784000A0E80C50A0E80C50B1F12001BFF4F7AF54
:10785000090728BFA0E80C5048BF0CC05DF804EB36
:10786000890028BF40F8042B08BF704748BF20F8A4
:10787000022B11F0804F18BF00F8012B7047000059
:1078800000487047040400207546FFF7F9FFAE4634
:1078900005006946534620F00700854618B020B51C
:1078A000F8F7D2FCBDE820404FF000064FF000078B
:1078B0004FF000084FF0000B21F00701AC46ACE898
:1078C000C009ACE8C009ACE8C009ACE8C0098D4605
:1078D000704710B50446AFF300802046BDE8104065
:1078E000F8F79DBC4FF0013C50F8042B51F8043BD5
:1078F0009A4221D1A2EB0C03934313EACC1317D184
:1079000050F8042B51F8043B9A4215D1A2EB0C031A
:10791000934313EACC130BD150F8042B51F8043BDA
:107920009A4209D1A2EB0C03934313EACC13DBD0A8
:107930004FF00000704700BFD01A01BAB1FA81F1D0
:1079400001F0180122FA01F0CB40C1F12001DBB2B5
:10795000C0B2C01A2CFA01F3D11A914311EAC31133
:10796000E6D170475FEA400C08BF91F0000F4FEA84
:107970008C234FEAC12243EA51514FEA1C5018BFF1
:1079800000F5F0404FEA300018BF41F000415FEAD7
:107990006C5C00F02980BCF1FF3F08BF40F08040E4
:1079A0007047130C06BF12044FF0100C4FF0000C80
:1079B000130E04BF12020CF1080C130F04BF1201C6
:1079C0000CF1040C930F04BF92000CF1020CD30FC6
:1079D00004BF52000CF1010C11464FF00002A0F15F
:1079E0001F00A0EB0C00704711F0004F08BF70475C
:1079F00031F000413FF4D5AF0B0C06BF09044FF046
:107A0000100C4FF0000C0B0E04BF09020CF1080C17
:107A10000B0F04BF09010CF1040C8B0F04BF89008C
:107A20000CF1020CCB0F04BF49000CF1010CCCF19E
:107A30002003A0EB0C0022FA03F302FA0CF241EA55
:107A4000030100F10100704720F07F4C80EA030041
:107A500023F07F47ACEB070303F57C5300F00040B5
:107A600003F1FF032DE980494FEA154B09B44FEAB2
:107A7000144325EA0B4E24EA03480FF2042606EBD2
:107A8000132749083E785FEA320203FB0667C7F511
:107A9000000707FB06F64FEA54374FEAD64606F1D1
:107AA000020607FB066CCCF1005C4FEA1C472CEA8F
:107AB000074C07FB06F40CFB06F504EB15464FEAF2
:107AC000961634BF00204FF000404FEAD13706FB36
:107AD00007FC4FEA1C4C0CFB0BF7D21B03FB0CF70B
:107AE00061EB07010CFB0EF7B0EB074072EB17429E
:107AF0000CFB08F734BFA2EB0742B2EB074261EB85
:107B000017414FEA0C444FEA910706FB07FC4FEA86
:107B10001C4C0CFB0BF7B0EBC74072EB573203FB6E
:107B20000CF734BFA2EBC742B2EBC74261EB57314F
:107B30000CFB0EF7B0EBC70072EB57720CFB08F7AB
:107B400034BFA2EBC702B2EBC70261EB5771039FD0
:107B50004FEA816141EA921104EBCC044FEAD1373C
:107B60004FEA826206FB07FC42EA90124FEA80600D
:107B70004FEA1C4C0CFB0BF7D21B03FB0CF761EB21
:107B800007010CFB0EF7B0EB074072EB17420CFB42
:107B900008F734BFA2EB0742B2EB074261EB174193
:107BA0004FEA8C554FEA910704EB9C2406FB07FC37
:107BB0004FEA1C4C0CFB0BF7B0EBC74072EB573293
:107BC00003FB0CF734BFA2EBC742B2EBC74261EB39
:107BD00057310CFB0EF7B0EBC70072EB57720CFB82
:107BE00008F734BFA2EBC702B2EBC70261EB5771D3
:107BF00015EB4C254FEA816141EA92114FEA82620E
:107C00004FEAD13742EA901206FB07FC44F1000428
:107C10004FEA80604FEA1C4C0CFB0BF7D21B03FBB6
:107C20000CF761EB07010CFB0EF7B0EB074072EBB2
:107C300017420CFB08F734BFA2EB0742B2EB074236
:107C400061EB174115EB1C154FEA813141EA924176
:107C50004FEA823242EA90424FEA80304FEA0C7695
:107C600044F1000448EA03434EEA0B484FF0000E8B
:107C7000B2EB080C71EB030724BF624639464EEBAA
:107C80000E0E4FF0000B0018524149414BEB0B0B0D
:107C9000B2EB080C71EB03077BF1000B24BF6246CB
:107CA00039464EEB0E0E4FF0000B00185241494181
:107CB0004BEB0B0BB2EB080C71EB03077BF1000BEA
:107CC00024BF624639464EEB0E0E51EA020718BF3A
:107CD00046F0010616EB0E7655F1000254F1000154
:107CE00003D5BDE88901BDE80088BDE88901BDE88C
:107CF0000048B619524141EB0101A3F1010370475D
:107D000080807F7E7D7C7B7A7978777676757473D8
:107D1000727171706F6E6E6D6C6C6B6A6A69686897
:107D2000676666656464636362616160605F5F5E2D
:107D30005E5D5D5C5C5B5B5A5A59595858575756A3
:107D40005655555554545353525252515150505008
:107D50004F4F4F4E4E4D4D4D4C4C4C4B4B4B4A4A5A
:107D60004A4949494848484747474746464645459E
:107D700045444444444343434342424242414141D7
:107D8000002B26D4770021D01CB54FEA370703B467
:107D90004FF010004FF010014FF000000FBCBDE895
:107DA00010400BF1010BBBF1010F08BF5FEA170791
:107DB00022BF12F1010211F101014FF0004143F124
:107DC000000300F0004043EA00007047F9D3570871
:107DD000DAE746EA064613F1400F4FEA16461FDD82
:107DE00013F1200FDFBF16430A46002120335B4208
:107DF000C8D0C3F1200746EA064602FA07F74FEA61
:107E0000164646EA0706C3F1200722FA03F201FAF2
:107E100007F721FA03F14FF0000342EA0702B1E746
:107E200046EA020646EA06464FEA164646EA0106D2
:107E3000BCBF46EA0646360C4FF000034FF0000286
:107E40004FF000019EE72DE9C048934630B491E819
:107E5000380007C831EA400C48BF34EA430C03D568
:107E6000FFF7F2FDFFF78CFFF0BCBDE800882DE9BD
:107E7000C048934630B491E8380007C810F0804FEE
:107E800008BF13F0804F03D100F005F8FFF778FF2B
:107E9000F0BCBDE8008820F07F4780EA030023F0B3
:107EA0007F4C07EB0C03A3F57C5300F00040A3F1DB
:107EB000FE0392F0000F00F0B38095F0000F00F089
:107EC00077802DE901494FEA11404FEA144621EA33
:107ED000004800FB06FC24EA064708FB06F607FB01
:107EE00008F800FB07F718EB06484CEB164C4FEA76
:107EF000124B18EB07484FEA15464CEB174022EAA5
:107F00000B4E0BFB06FC25EA06470EFB06F607FBAD
:107F10000EFE0BFB07F71EEB064E4CEB164C4FF01C
:107F200000061EEB074E4CEB174B18EB0B0840F10D
:107F3000000018EB0E0B58EB000840F100008F1A00
:107F40004FF000013CBFC943661B14BFB5EB040CE6
:107F500000213CBFC943F61B4FEA17444EEA8E0E80
:107F600027EA04454FEA1C4704FB07622CEA074C4A
:107F700005FB07F70CFB05F604FB0CFC16EB0746AC
:107F800042EB174216EB0C4642EB1C421BEB06067B
:107F900058EB0202414146EA9E0601D5BDE801893F
:107FA000B619524141EB0101A3F10103BDE801897A
:107FB0004FEA14454FEA114724EA054621EA074CE7
:107FC00005FB07F406FB07F70CFB06F105FB0CFCB1
:107FD00011EB074144EB17444FEA124711EB0C41F8
:107FE00044EB1C4422EA074C05FB07F206FB07F7AB
:107FF0000CFB06F605FB0CFC16EB074642EB1742A2
:1080000016EB0C4642EB1C456A1854F1000148BFC0
:108010007047B619524141EB0101A3F101037047CA
:1080200095F0000F37D04FEA11424FEA144721EA8A
:10803000024624EA074C02FB07F106FB07F70CFB9C
:1080400006F402FB0CFC14EB074441EB17414FEA2A
:10805000154714EB0C4441EB1C4125EA074C02FB8D
:1080600007F506FB07F70CFB06F602FB0CFC16EB0C
:10807000074645EB174516EB0C4645EB1C4212191B
:1080800051F1000148BF7047B619524141EB01015F
:10809000A3F1010370474FEA14454FEA114724EA60
:1080A000054621EA074C05FB07F106FB07F70CFB29
:1080B00006F24FF0000605FB0CFC12EB074241EB09
:1080C000174112EB0C4251EB1C4148BF704792180C
:1080D00041EB0101A3F101037047490050EAC120BF
:1080E00018BF04204A0D18BF40F0010040F2FF7293
:1080F000B2EB515F08BF40F00200012808BF052025
:1081000070472DE9F0414F1E00EBC7010446D1E94D
:10811000000115461E4637F006020DD02A463346AA
:1081200000F092FC7F1E04EBC703D3E9002300F0AC
:108130006BFA37F00602F1D1022F25D0042F13D0AD
:10814000062F18BFBDE8F0812A46334600F07CFCBC
:10815000D4E90A2300F058FA2A46334600F074FCAA
:10816000D4E9082300F050FA2A46334600F06CFCAC
:10817000D4E9062300F048FA2A46334600F064FCAE
:10818000D4E9042300F040FA2A46334600F05CFCB0
:10819000D4E9022300F038FA2A46334600F054FCB2
:1081A000D4E90023BDE8F04100F02EBA012201F02D
:1081B0001CBA00F029BA0000024A0020110701F0A1
:1081C00014BA000001FDFFFF30380A2801D2012057
:1081D00070470020704700002DE9F84F04460D4617
:1081E00021F0004000917349814211DC72498842BC
:1081F00001DC06D12CB120462946BDE8F84FFFF737
:10820000D5BF6E48002DCCBF6D496E49BDE8F88FD3
:108210006D49814211DD6D498142D8BF4FF0FF3673
:108220006DDD20462946FFF758FF042808BFFFF7F9
:10823000C3FF20462946BDE8F88F6549654F25F004
:108240000045814233DD6449814219DD0026324612
:108250004FF080432046294600F0D6F980468A46F2
:1082600001222046294601F0C0F900223B4600F0D9
:10827000F5FC4246534600F077FA04460D463EE0D0
:1082800001260022BA463B462046294600F0BCF9AA
:1082900080460F46002253462046294600F0DEFC69
:1082A00042463B4600F060FA04460D4627E04B4943
:1082B00081421BDDDFF828A102260022534620461A
:1082C000294600F0C1FB00223B4600F09DF98046A4
:1082D0000F46002253462046294600F0BFFC424686
:1082E0003B4600F041FA04460D4608E003262246CC
:1082F0002B4600203B4900F037FA04460D46224643
:108300002B461046194600F09FFB8B4682460246DC
:108310000B4600F099FB07460246334888460B4659
:1083200006217844FFF7EDFE52465B4600F08CFBD9
:1083300082462E488B463A46434605217844FFF74D
:10834000E0FE3A46434600F07FFB02460B46002E15
:10835000504659460CDA00F057F922462B4600F0F9
:1083600073FB01B022462B46BDE8F04F00F06ABC1B
:1083700000F04AF922462B4600F066FB1C4A7A447C
:1083800002EBC603D3E9002300F068FC22462B462B
:1083900000F064FC174A7A4402EBC603D3E90023D9
:1083A00000F050FC009A002AB8BF81F00041BDE8FF
:1083B000F88F0000000010440000F07F182D445496
:1083C000FB21F93FFB21F9BF0000DC3F0000203E0C
:1083D0000000F33F0000F03F0000E63F0080034054
:1083E0000000F83F0000F0BF1A280000D827000066
:1083F000762700003E2700002DE9F04D9446CCF191
:10840000000423F000464CEA0404524F46EAD474B8
:108410009A46884621F00042BC4206D8454240EACE
:10842000050442EAD474BC4204D9BDE8F04D62466A
:10843000FFF7BFBEAAF14055A5F17F6555EA0C04D0
:108440000BD0022404EAAA74434DDFF810E144EA99
:10845000D87452EA000B04D00CE0BDE8F04DFFF7F1
:10846000BBBE002C14BF012CBDE8F08D022C30D017
:10847000032C32D056EA0C0B0AD0BE4220D1BA42AD
:1084800009D126F0804622F080423346114617E09B
:1084900000291ADB25E0DFF8C8B0FB44002C04BF3C
:1084A000DBE90001BDE8F08D012C02BFDBE9000132
:1084B00081F00041BDE8F08D022C0AD0032C0CD0D5
:1084C000BA4212D1B8F1000F0BDA23482549BDE8B2
:1084D000F08D28462449BDE8F08D28467146BDE858
:1084E000F08D1D482149BDE8F08D921B12153C2AE4
:1084F000C4BF19481D490EDCBAF1000FBEBF12F10E
:108500003C0F0020014606DB624600F02DF921F009
:108510000041FFF761FE002C08BFBDE8F08D012C83
:1085200004BF81F00041BDE8F08D114A114B022CCF
:1085300007D000F093FB2A46BDE8F04D0A4B00F04F
:108540008DBB00F08BFB2A46BDE8F04D064B00F0DA
:1085500079BB00000000F07F182D4454FB2109C0B6
:10856000D2260000FB21F9BFFB210940FB21F93F86
:10857000075C143326A6A13C10B500290AD0087860
:10858000002807D005487844FFF7ACF9002801D04F
:10859000002010BD0248784410BD0000F6260000FF
:1085A000EE26000021F00042A2F16052B2F5801FD9
:1085B00001F0004328BFD2F17F6C0BD95FEA001CA9
:1085C00043EAC20242EB507018BF704728BF20F048
:1085D00001007047B2F5801FBCBF184670474FEAD4
:1085E000410C1CF5001F02D2084600F014BF70B504
:1085F00000F0D4FA00000089FFF7F6BF4FF000400A
:10860000A0F580007047000010B591EA030F48BF45
:1086100083F0004300F12A83841A71EB030C05D226
:10862000121943EB0C03001B61EB0C01DFF824E192
:108630004FEA1154A4EB135C1EEA430F18BF9EEAE5
:10864000445F73D023EA0E03DCF1200E21EA0451CB
:1086500043F4801332D322FA0CFE10EB0E0023FAFF
:108660000CFE41EB0E01CCF1200E03FA0EFE10EBD6
:108670000E0051F10001B1F5801FCCF1200E32D275
:1086800001EB045112FA0EF2BDE8104058BF7047DA
:10869000401C38BF5FEA420218BF7047002814BF71
:1086A00020F0010041F100014FEA410313F5001FE2
:1086B00038BF7047A1F1C04100F0BEBA012A43EBB8
:1086C0000302ACF1200CDCF11F0E32BF4FF0000EA4
:1086D00023FA0CF310EB030041EB0451B4EB115FF0
:1086E000D0D0A1EB045101F5801149085FEA3000B8
:1086F00001EB04510ED350F1000038BF12FA0EFE08
:1087000008D1BDE81040C9E7401C38BF5FEA42020B
:10871000CAD1C3E7BDE810404FEA410313F5001F7B
:1087200038BF7047A1F1C04100F086BA9EEA445FAD
:1087300008D011EA5E0FBDE8104004BF01F000410F
:1087400000207047BDE8104070B500F027FA00BF68
:1087500064FBBE3E0000E0FF02494FF0000000F065
:1087600012BF00BF0000F87F2DE9C04130B4DFF830
:10877000A0C23CEA111418BF3CEA131400F0EC80CC
:1087800081EA03051CEA111444EAD57418BF1CEAF7
:10879000131500F0C780A4EB05044FF0004545EA2F
:1087A000C12145EAC32341EA505143EA525304F13F
:1087B0007F74994204F500344FEAC0204FEAC22288
:1087C00008BF904200F09C804FEA13650FF24016FC
:1087D000765D4FEA134506FB05F7C7F1807706FB88
:1087E00007F74FEAD737A7FB03687642C8F580380A
:1087F000A7FB06CE38BFA8F1010807FB08E64FF03B
:10880000000EA6FB028CE6FB03CEDCF1000CCEF1E1
:10881000004E38BFAEF1010EA6FB0C584FF000071A
:108820004FF00005E6FB0E87A1FB08C6A0FB07CEB4
:1088300016EB0E0645F10005E1FB076515F1E04E6C
:108840007EBFA4F580345FEA46066D4116F18007CD
:1088500045F100054FEA17274FEA066647EA056724
:10886000A6F1DE46B6F1805F4FEA15251FD93846DE
:1088700024F0010C05EBC471BCF1FE6F01EB0C118F
:1088800002D8F0BCBDE8008124425CBF01F5801E27
:108890009EEAC47F02D4F0BCBDE80081244238D4F3
:1088A000F0BCA1F1C041BDE8004100F0C5B94FEAFC
:1088B000D22242EA43524FEAD323A7FB02864FEA71
:1088C000D02040EA415007FB03661EEA0E0F4FEA34
:1088D000D12105FB026658BFA6EB0056B6EB005649
:1088E0004FEA520E4EEAC37E18EB0E0E56EB530EB5
:1088F000BDD518EB02085E417F1C55F10005B6E7B7
:108900004FF480154FF000074FF000064FF00008BD
:10891000ADE7F0BC4FF0000001F1C04101F00041B3
:10892000BDE8008111EA0C1F0CEA131500D00CE021
:1089300013EA0C1F00F025804FF00000F0BC81EA24
:10894000030101F00041BDE80081F0BCBDE8004139
:1089500081EA030100F070B9F0BCBDE8004170B5D8
:1089600000F01CF9097EFC3E00F007B881EA030123
:108970004FF0000001F00041704781EA030100F070
:108980005BB9F0BCBDE800414FF0000021497047E1
:10899000FFFDFBF9F7F5F4F2F0EEEDEBE9E8E6E4C4
:1089A000E3E1E0DEDDDBDAD8D7D5D4D3D1D0CFCD4B
:1089B000CCCBCAC8C7C6C5C4C2C1C0BFBEBDBCBB84
:1089C000BAB9B8B7B6B5B4B3B2B1B0AFAEADACAB7F
:1089D000AAA9A8A8A7A6A5A4A3A3A2A1A09F9F9E59
:1089E0009D9C9C9B9A99999897979695959493930B
:1089F000929191908F8F8E8E8D8C8C8B8B8A8989A2
:108A00008888878786858584848383828281818024
:108A10000000FF070000F87F10F0004248BF40420E
:108A2000B0FA80F310FA03F10AD0C3F11D0303F585
:108A300080634FEA415002EB035202EBD1217047B1
:108A40004FF0000070470000DFF848C170B51CEA25
:108A5000111E1EBF1CEA13159EEA0C0F95EA0C0F9F
:108A600000F06F8081EA030423EA4C134EEAD47EBF
:108A700021EA4C1141F4801143F48013AE44A1FB70
:108A8000024CA0FB0365AEF17F7E361955EB0C0559
:108A9000A1FB034C4CF10003A0FB021C16EB0C06DF
:108AA000654153F10003094218BF46F0010613F473
:108AB000007F0BD14FEA03314FEA0530340341EA1E
:108AC000155140EA16506FF003020AE04FEAC32145
:108AD0004FEAC520F40241EA555140EA56506FF082
:108AE000020202EB2E4201EB025585EACE710AD05A
:108AF0005FEA440C18BF24F0004450F1000041F13B
:108B0000000120EAD47040F2FE7C624500D270BDC4
:108B1000A84214BF4FF080444FF04044002E08BFDD
:108B20000024BEF1806FA8BFA1F1C041BDE8704034
:108B300080F282804FF0000001F1C04101F000415D
:108B400070479EEA0C0F0CEA131518BF95EA0C0F3C
:108B500006D04FF0000081EA030E0EF0004170BD18
:108B600000F01CF88900013E00F007B800F009B8D9
:108B70004FEA430C5FEA5C5C08D081EA030100F035
:108B80005BB84FEA410C5FEA5C5CF6D14FF0000045
:108B9000014970470000FF070000F87F0EF1020E48
:108BA0002EF0030E5EF8046B364205D4012A43EB27
:108BB000030515F5001F12D8012841EB010C1CF527
:108BC000001F0CD80ED14FEAD17C15F5001F0CEB1D
:108BD0004C0C0CF1020C08BF4CEBD37C04E04FF0C2
:108BE000080C01E04FEAD37C0CEB4C0526FA05F6A5
:108BF00006F00706B6F1040C06D20EEB860CBDE8B3
:108C000070404CF0010C6047DFE80CF0090B0202E9
:108C10004FF000414FF00000A1F5002170BD194652
:108C20001046012851EB010418BFD4F5001484BF8D
:108C3000002001F0004170BD0808A0F500114FEAC6
:108C40003101704791EA030F10B581F000413FF503
:108C5000E3AC83F0004300F009B8000010B591EADE
:108C6000030F48BF83F000433FF5D6AC841A71EB85
:108C7000030C07D212198CF0004C43EB0C03001BC1
:108C800061EB0C01DFF8A4E14FEA1154A4EB135C93
:108C90001EEA430F18BF9EEA445F00F0B08023EA4B
:108CA0006E03524221EA0451C3EB6E0338BF5B1ED0
:108CB000DCF1200E25D322FA0CFE10EB0E0043FA55
:108CC0000CFE41EB0E01CCF1200E03FA0EFE10EB70
:108CD0000E0051F10001CCF1200E29D412FA0EF24F
:108CE00001EB0451BDE8104058BF7047401C1CBF49
:108CF000B2F1004F704700280CBF491C20F0010062
:108D0000704712EB020E43EB030218BF4FF0010E47
:108D10004EEA4202ACF1200CDCF11E0E54D943FAAB
:108D20000CFE10EB0E0051F1FF31CCF11E0ED5D52B
:108D30000EF1010E12FA0EFE404141EB010101EB72
:108D4000445C5FEA5C5C10D910EBDE7001EB04510F
:108D500038BFBEF1004FBDE8104018BF7047002873
:108D60000CBF491C20F00100704730D24FEAD42CD0
:108D700011F5001124F400641BD0B1FA81F20B3A12
:108D8000A41AA41ED2F12003914030FA03F3194330
:108D9000904001EBCC71002C01EB0451BDE8104078
:108DA000A8BF704701F1C0414FF0000001F0004141
:108DB0007047B0FA80F310FA03F100D110BDE41A45
:108DC000173C4805C90AE4E701EB045110BD4910FE
:108DD00001EB0451BDE810404FEA300002E04FF0D3
:108DE000000170474A0008BF0042F8D0B2F5001FEA
:108DF00028BF704701F000414FF0000070479EEA25
:108E0000445F07D011EA5E0FBDE8104004BF0021A7
:108E100000207047BDE8104070B5FFF7BFFE00BFEF
:108E200040DFF63E83F00041104670470000E0FF4F
:108E300043004FEAD30C4FEA3C0C43401FBF4007AE
:108E40000CF1605113F0FE4F70471CF0006F03D11E
:108E500000200CF0004170470CF0004343EA5070D2
:108E600010B540EACC0000F090FA00BF000000927C
:108E70004FEA0001FFF7E0BE4FF000414FF0000065
:108E8000A1F500217047000090EA010F48BF81F072
:108E9000004100F10883421A3CBF801A89184FEA4A
:108EA000D0524FF07F4C1CEA410FA2EBD15318BFB8
:108EB0009CEA026F00F03B804FF0004C4CEA00202F
:108EC0004CEA012121FA03FC10EB0C0C1ED202F13A
:108ED000FF325FEA1C2040EBC25038BF70471CF0E5
:108EE0007F0F4FEA400C18BFBCF17F4F38BF70476F
:108EF000C3F12003994008BF20F00100BCF17F4F6F
:108F000038BF7047A0F1C04000F085BA4FEA3C007E
:108F1000000A40EBC25028BF1CF0FF0F4FEA400C84
:108F2000E6D018BFBCF17F4F38BF7047EAE79CEA34
:108F3000026F05D010EA5C0F08BF00F000407047D8
:108F400010B500F022FA00BF64FBBE3E401058BFCF
:108F5000C0F14040491058BFC1F140418142EFF398
:108F6000008070474FF47F0C1CEAD0121EBF1CEA31
:108F7000D11392EA0C0F93EA0C0F00F0858090EA6F
:108F8000010F48BF42F4807240F4000C41F400002D
:108F90002CF07F4120F07F4000B58142A2EB03021C
:108FA0000FF2081CACEB504EC0F100009EF800E040
:108FB0004FEA4E0E00FB0EFC38BF49004FEA2C1C56
:108FC00002F5FA020CFB0EF34FEACE1E4FEA112C0B
:108FD0004FEAC1210EEB635E42EB22420EFB0CFC1A
:108FE0004FEA1C5300FB03114FEA112C4FEA0131E9
:108FF0000EFB0CFC4FEADC4C00FB0C11C14228BFFD
:1090000009184CEB03335DF804EB10EB410143EB23
:10901000C250B2F57C0F38BF704729D512F0F00F5F
:109020001CBF00F1C04000F0004070470081828307
:109030008485868788898B8C8D8E8F919293959667
:1090400097999A9C9D9FA0A2A3A5A7A8AAACAEB0F1
:10905000B2B3B5B7B9BCBEC0C2C5C7C9CCCED1D4F6
:10906000D7D9DCDFE2E6E9ECF0F3F7FAFE00000026
:109070004FEA400C0CF1807CBCF17E4F28BF70475A
:10908000B0F1C04000F0C7B990EA010F0CEAD1136B
:1090900048BF42F48072624538BF634507D213F47B
:1090A0007F0F16D080EA010000F00040704710B535
:1090B00000F06BF9097EFC3E00F005B880EA010083
:1090C00000F00040704780EA010000F0004000F02E
:1090D000A2B912F47F0F04BF0248704780EA010072
:1090E00000F099B90000C07F50EA010C00F1138034
:1090F0001CF5000F58BFBCF5000F01D48842704723
:1091000007D710F5000F58BF11F5000F15D488428E
:109110007047894270471CF5000F04D5BCF5000F5D
:10912000F7D5814270474FF0807C1CEB400F38BF71
:109130001CEB410F01D28142704710B500F025F9B8
:10914000922449004FF000504FF08051FFF7FEBECF
:1091500041000B0ED3F19E0208D950F400034FEAF0
:10916000032323FA02F048BF4042704710B500F0D5
:109170000CF900BF49922480002070476FF0004234
:1091800082EA200070470000C10DD1F19E0206DB8B
:109190004FEA002343F0004323FA02F070470042F5
:1091A00007D54FEA4001B1F1FE4F02D24FF0000067
:1091B000704710B500F0E9F849922480002070470C
:1091C0006FEA20007047000010F0004148BF4042A5
:1091D000B0FA80F310FA03F2C3F19D030BD051EA09
:1091E000C35101EB1220530638BF704700F1010054
:1091F00008BF20F001007047B0FA80F310FA03F2C4
:10920000C3F19D030AD0D90501EB1220530638BFE4
:10921000704700F1010008BF20F001007047000016
:1092200050EA010C00F113801CF5000F58BFBCF58B
:10923000000F01D48842704707D710F5000F58BFC0
:1092400011F5000F15D488427047894270471CF50C
:10925000000F04D5BCF5000FF7D5814270474FF0E1
:10926000807C1CEB400F38BF1CEB410F01D28142C8
:10927000704710B500F089F8922449004FF0005073
:109280004FF08051FFF762BE4FF47F0C1CEAD01202
:109290001EBF1CEAD11392EA0C0F93EA0C0F00F0E8
:1092A000478090EA010F48BF42F480724FF0004CB3
:1092B0004CEA00204CEA012102EB0302A0FB01135F
:1092C000A2F50002002918BF43F001035B0028BF8C
:1092D0004FEA330342EB22425FEA132C4CEBC250BD
:1092E0002EBFBCEB436FB2F57C0F70474FEA036CA7
:1092F000BCF1004F08BF20F00100B2F57C0F38BF71
:1093000070470BD582F0FF0212F5803FC8BF70474F
:1093100000F1C040D8BF00F00040704700F5000CDD
:109320005FEA4C0C48BF7047B0F1C04000F073B822
:1093300090EA010F0CEAD11348BF42F480726245F3
:1093400038BF634504D280EA010000F00040704756
:1093500010B500F01AF800BF8900013E00F007B810
:1093600000F009B85FEA410C5FEA1C6C08D080EAA3
:10937000010000F050B85FEA400C5FEA1C6CF6D1C7
:109380004FF00040A0F5800070470EF1020E2EF065
:10939000030E5EF8044B244204D44FEA4102B2F1BA
:1093A0007F4F11D84FEA4003B3F17F4F0CD80ED155
:1093B0004FEAD07CB2F17F4F0CEB4C0C0CF1020C5D
:1093C00008BF4CEBD17C04E04FF0080C01E04FEA01
:1093D000D17C0CEB4C0324FA03F404F00704B4F141
:1093E000040C06D20EEB840CBDE810404CF0010CCE
:1093F0006047DFE80CF0070802024FF00040A0F5DC
:10940000800010BD0846420018BFD2F1807288BFAC
:1094100000F0004010BDFF2141EAD050C005704768
:1094200051EA000C00F113801CF5000F58BFBCF589
:10943000000F01D48142704707D711F5000F58BFC4
:1094400010F5000F15D481427047894270471CF512
:10945000000F04D5BCF5000FF7D5884270474FF0D8
:10946000807C1CEB410F38BF1CEB400F01D28842BF
:10947000704780EA010081EA000180EA0100FFF7FD
:10948000F8BE80F0004090EA010F7FF504AD81F056
:10949000004100F008B8000090EA010F48BF81F0D9
:1094A00000413FF5F8AC421A04D882F00042A0EB2C
:1094B000020011444FEAD0524FF07F4C1CEA410F9A
:1094C000A2EBD15318BF9CEA026F4AD04FF0004C78
:1094D0004CEA00204CEA012121FA03FCB0EB0C0C11
:1094E0000FD412F0FE0F36D05FEA4C001DD50012EB
:1094F00040EBC25038BF70471CF03F0F18BF704799
:109500000BE0A2F101025FEA1C2040EBC25038BF21
:1095100070471CF07F0F18BF7047C3F120039940BC
:1095200014BF401E20F00100704780084FEA12234C
:1095300008BF7047B0FA80FCA2EB0C02CCF1280CFB
:1095400060FA0CF093EA122F04BF00EBC250704790
:109550004FEAC3707047130A5FEADC1008BF704718
:10956000F6E79CEA026F04D010EA5C0F08BF002007
:10957000704710B5FFF709FF40DFF63E81F000406D
:109580007047FDF7D1BE0CF00F03092B08BF082070
:1095900000F059800A2B0BD0082B18BF704708BF6A
:1095A0001CF0400F0AD04FF000004FF00001704750
:1095B0001CF0400F18BF4FF0004070471CF0100F18
:1095C00008D020F0704300F07F4242EAD3014FEA16
:1095D0004370704700F0604021F07F4242EA000291
:1095E00001F07F4040EA727070474FF0FF0C4CF47E
:1095F000E06C1CEA11531CBF9CEA030C9445C2BFEB
:10960000DA4201EB02517047002B0DD0BCF1000F84
:109610000FD0002A01F00041A4BF41F0E04141F029
:109620007F614FF00000704701F000414FF00000F3
:10963000704750EA01334FF09B0C18BF4CF0806C20
:109640007FF48AA870471CF4801F11D01CF4E02F0F
:1096500003D06FEACC31490070474FF04050EFF330
:10966000008222F0704242EA000282F300887047D2
:109670004FF0000070470000000000000000002FC5
:10968000000000000700070000147F147F1400246E
:109690002A7F2A120062640813230036495522509B
:1096A00000000503000000001C22410000004122D0
:1096B0001C000014083E08140008083E08080000BA
:1096C00000A06000000808080808000060600000B2
:1096D000002010080402003E5149453E0000427F30
:1096E0004000004261514946002141454B3100187C
:1096F00014127F10002745454539003C4A4949303E
:1097000000017109050300364949493600064949F7
:10971000291E000036360000000056360000000802
:1097200014224100001414141414000041221408DF
:1097300000020151090600324959513E007C1211C4
:10974000127C007F49494936003E41414122007F59
:109750004141221C007F49494941007F0909090113
:10976000003E4149497A007F0808087F0000417F98
:109770004100002040413F01007F08142241007F4A
:1097800040404040007F020C027F007F0408107FB1
:10979000003E4141413E007F09090906003E41511A
:1097A000215E007F091929460046494949310001D7
:1097B000017F0101003F4040403F001F2040201F2B
:1097C000003F4038403F00631408146300070870EE
:1097D000080700615149454300007F4141000055A1
:1097E0002A552A55000041417F000004020102046D
:1097F000004040404040000001020400002054545A
:109800005478007F484444380038444444200038A9
:109810004444487F00385454541800087E0901021B
:109820000018A4A4A47C007F080404780000447DF0
:109830004000004080847D00007F1028440000002C
:10984000417F4000007C04180478007C0804047800
:1098500000384444443800FC2424241800182424EC
:1098600018FC007C080404080048545454200004E8
:109870003F444020003C4040207C001C2040201CF5
:10988000003C4030403C004428102844001CA0A06C
:10989000A07C004464544C441414141414140000A8
:1098A00000000000000000000000000000000000B8
:1098B00000F800000000000000333000000000103D
:1098C0000C06100C0600000000000000000040C064
:1098D0007840C0784000043F04043F040400007056
:1098E00088FC08300000001820FF211E0000F0084E
:1098F000F000E018000000211C031E211E0000F0F3
:109900000888700000001E2123241927211010163A
:109910000E00000000000000000000000000000039
:1099200000E01804020000000007182040000002B8
:109930000418E0000000004020180700000040402C
:1099400080F0804040000202010F0102020000008E
:1099500000F0000000000101011F010101000000F2
:1099600000000000000080B0700000000000000057
:1099700000000000000000010101010101010000E0
:109980000000000000000030300000000000000077
:10999000000080601804006018060100000000E06C
:1099A00010080810E000000F102020100F00001019
:1099B00010F8000000000020203F20200000007070
:1099C0000808088870000030282422213000003068
:1099D0000888884830000018202020110E00000060
:1099E000C02010F8000000070424243F240000F8E1
:1099F0000888880808000019212020110E0000E0C6
:109A0000108888180000000F112020110E00003867
:109A10000808C83808000000003F0000000000707F
:109A2000880808887000001C222121221C0000E008
:109A300010080810E0000000312222110F00000081
:109A400000C0C00000000000003030000000000036
:109A500000800000000000008060000000000000A6
:109A6000804020100800000102040810200040403F
:109A70004040404040000404040404040400000882
:109A80001020408000000020100804020100007037
:109A900048080808F0000000003036010000C0301F
:109AA000C828E810E0000718272423140B00000042
:109AB000C038E0000000203C23020227382008F8CC
:109AC000888888700000203F202020110E00C030C0
:109AD000080808083800071820202010080008F897
:109AE00008080810E000203F202020100F0008F890
:109AF0008888E8081000203F20202320180008F85C
:109B00008888E8081000203F200003000000C030D3
:109B100008080838000007182020221E020008F854
:109B200008000008F808203F210101213F2000081B
:109B300008F8080800000020203F20200000000056
:109B40000808F8080800C08080807F00000008F83E
:109B500088C028180800203F20012638200008F877
:109B6000080000000000203F20202020300008F8DE
:109B7000F800F8F80800203F003F003F200008F8F8
:109B800030C00008F808203F200007183F00E01010
:109B900008080810E0000F10202020100F0008F81F
:109BA00008080808F000203F210101010000E01032
:109BB00008080810E0000F18242438504F0008F857
:109BC000888888887000203F2000030C30200070B7
:109BD0008808080838000038202121221C001808B5
:109BE00008F8080818000000203F2000000008F8CE
:109BF00008000008F808001F202020201F00087817
:109C0000880000C83808000007380E010000F80876
:109C100000F80008F800033C0700073C03000818A0
:109C200068808068180820302C03032C3020083806
:109C3000C800C83808000000203F200000001008BD
:109C40000808C83808002038262120201800000005
:109C500000FE020202000000007F40404000000CB5
:109C600030C000000000000000010638C000000203
:109C70000202FE000000004040407F0000000000A3
:109C800004020202040000000000000000000000C6
:109C900000000000000080808080808080800002C2
:109CA00002040000000000000000000000000000AE
:109CB0008080808000000019242222223F2008F8A2
:109CC000008080000000003F112020110E000000E5
:109CD000008080800000000E112020201100000074
:109CE00000808088F800000E112020103F20000026
:109CF000808080800000001F22222222130000802A
:109D000080F0888888180020203F20200000000074
:109D1000808080808000006B94949493600008F8A9
:109D2000008080800000203F210000203F20008034
:109D30009898000000000020203F20200000000034
:109D400000809898000000C08080807F000008F8A4
:109D5000000080808000203F24022D302000000879
:109D600008F8000000000020203F20200000808034
:109D7000808080808000203F20003F20003F808046
:109D8000008080800000203F210000203F20000054
:109D9000808080800000001F202020201F00808005
:109DA00000808000000080FFA12020110E00000034
:109DB000008080808000000E112020A0FF80808025
:109DC00080008080800020203F21200001000000D2
:109DD00080808080800000332424242419000080A7
:109DE00080E0808000000000001F202000008080B4
:109DF000000000808000001F202020103F20808075
:109E000080000080808000010E3008060100808004
:109E10000080008080800F300C030C300F00008029
:109E20008000808080000020312E0E312000808054
:109E300080000080808080818E7018060100008084
:109E40008080808080000021302C222130000000A2
:109E50000000807C020200000000003F4040000043
:109E60000000FF00000000000000FF0000000002F2
:109E7000027C800000000040403F0000000000061F
:109E800001010202040400000000000000000000C4
:109E90006800000476005401F7FD000175191A0CE2
:109EA0006A231B1C1F207274433B4138393A6B6C88
:109EB000376F06246D6E70008300000000080000FC
:109EC0000001001832000500000020410000D242CD
:109ED000295C0F3E9A99993E3333733F295C0F3EBC
:109EE00000007000000000240000000200030000D9
:109EF00000650054FFEF0000FA80000B12820001A1
:109F0000030C30C30E8C8CE914D5400213710F8EF4
:109F10003883F8833000F883258EF8833000F88387
:109F2000FFFFFFFF0FFEA9D6240004001A8279A1CB
:109F30000000003CFFFF00000010000038836FA20B
:109F4000003E03304000000002CAE3093E800000EA
:109F50002000000000000000400000006000000041
:109F6000000C0000000C186E000006920A16C0DFFC
:109F7000FFFF0256FD8CD377FFE1C496E0C5BEAA71
:109F800000000000FFFF0B2B0000165700000359D4
:109F90004000000000001DFA00026C1D00000000DF
:109FA0003FFFDFEB003EB3B6000D227800002F3CF0
:109FB00000000000001942B5000039A20000B3659E
:109FC000D90E9FC91DCF4C34300000005000000056
:109FD0003BB67AE80064000000C800000000000002
:109FE000100000001000FA921000225E000D229F67
:109FF0000001000000320000FF46000063D40000B2
:10A000001000000004D6000004CC000004CC0000C6
:10A01000000010720000004000000000000000007E
:10A0200000060002000500070000000000640000B8
:10A030000000000000000005000500640020000092
:10A0400000000000000000000000400000000300CD
:10A0500000000032F8980000FF650000830F000048
:10A06000FF9BFC000000000000000000000000005A
:10A0700000000000000000000000000000000000E0
:10A0800000000000000000000000000000001000C0
:10A0900040000000000000060000B26A000200005C
:10A0A0000001FB830068000000D9FC007CF1FF8305
:10A0B0000000000000650000006403E80064002860
:10A0C000000000250000000016A0000000001000A5
:10A0D00000001000002F0000000001F4000010003C
:10A0E00000280000FFFF4581FFFFFA72000000001A
:10A0F00000000000004400050005BAC6004778A231
:10A100000000000100000000000006000000001434
:10A110000000254D002F706D000005AE000C02D030
:10A12000000000000000000000000000000000002F
:10A13000001B000000000000000000000000000004
:10A1400000640000000800000000000000000000A3
:10A1500000000000000000000000000000000000FF
:10A1600000000000000000000000000000000000EF
:10A1700000000000000000000000000000000000DF
:10A1800000000000000000000000000000000000CF
:10A1900000000000000000000000000000000000BF
:10A1A000001B00000000000000000000000E000E78
:10A1B00000000AC70004000000000032FFFFFF9CFF
:10A1C00000000B2B000000020000000100000064F2
:10A1D000FFE500000000000000000000000000009B
:10A1E000000000010000000000010000000000006D
:10A1F000000180000001800000018000002426D3BF
:10A200000000000000000000000600100096003C66
:10A21000000000000000000000000000000000003E
:10A220000C0A4E68CDCF770950166759C619CE82F1
:10A23000000000000000000000000000000000001E
:10A24000000000000000000017D784000300000099
:10A250000000000000000000C7938F9D1E1B1C190A
:10A2600000000000000000000000000000000000EE
:10A2700000000000000000000203188500004000FC
:10A2800000000003000000030000000000000000C8
:10A29000400000000000000000000000000000007E
:10A2A00000000000000000000000000000000000AE
:10A2B000000000000000000000000000000000009E
:10A2C00000000000677DDF7E72902E554CF6E68818
:10A2D000000000000000000000000000000000007E
:10A2E000D8DCB4B8B0D8B9ABF3F8FAB3B7BB8E9E2C
:10A2F000AEF132F51BF1B4B8B08097F1A9DFDFDF22
:10A30000AADFDFDFF2AAC5CDC7A90CC92C97F1A936
:10A3100089264666B28999A92D557DB0B08AA8963E
:10A32000365676F1BAA3B4B280C0B8A89711B283FA
:10A3300098BAA3F0240844106418B2B9B49883F111
:10A34000A329557DBAB5B1A38393F0002850F5B287
:10A35000B6AA839328547CF1B9A3829361BAA2DA96
:10A36000DEDFDB819AB9AEF5606870F1DABAA2DFA0
:10A37000D9BAA2FAB9A38292DB31BAA2D9BAA2F8A9
:10A38000DF85A4D0C1BBAD83C2C5C7B8A2DFDFDF04
:10A39000BAA0DFDFDFD8D8F1B8AAB38DB4980D35F5
:10A3A0005DB2B6BAAF8C96198F9FA70E161EB49ADF
:10A3B000B8AA872C547CBAA4B08AB691325676B229
:10A3C0008494A4C808CDD8B8B4B0F19982A82D550A
:10A3D0007D98A80E161EA22C547C92A4F02C5078C6
:10A3E000F184A898C4CDFCD80DDBA8FC2DF3D9BA14
:10A3F000A6F8DABAA6DED8BAB2B68696A6D0F3C860
:10A4000041DAA6C8F8D8B0B4B882A892F52C54881E
:10A4100098F135D9F418D8F1A2D0F8F9A884D9C7A1
:10A42000DFF8F883C5DADF69DF83C1D8F40114F1FE
:10A43000A8824EA884F311D182F5D992289788F189
:10A4400009F41C1CD884A8F3C0F9D1D99782F1294A
:10A45000F40DD8F3F9F9D1D982F4C203D8DEDF1AAA
:10A46000D8F1A2FAF9A88498D9C7DFF8F8F883C719
:10A47000DADF69DFF883C3D8F40114F198A8822EDB
:10A48000A884F311D182F5D992509788F109F41C70
:10A49000D884A8F3C0F8F9D1D99782F149F40DD83E
:10A4A000F3F9F9D1D982F4C403D8DEDFD8F1AD884D
:10A4B00098CCA809F9D98292A8F57CF1883ACF9472
:10A4C0004A6E98DB6931DAADF2DEF9D88795A8F2E9
:10A4D00021D1DAA5F9F417D9F1AE8ED0C0C3AE827E
:10A4E000C684C3A88595C8A588F2C0F1F4010EF111
:10A4F0008E9EA8C63E56F554F18872F40115F19867
:10A5000045856EF58E9E0488F142985A8E9E068887
:10A5100069F4011CF1981E1108D0F504F11E970290
:10A5200002983625DBF9D985A5F3C1DA85A5F3DFD5
:10A53000D88595A8F309DAA5FAD88292A8F578F11A
:10A54000881A849F26889821DAF41DF3D8879F39CA
:10A55000D1AFD9DFDFFBF9F40CF3D8FAD0F8DAF990
:10A56000F9D0DFD9F9D8F40BD8F3879F39D1AFD917
:10A57000DFDFF41DF3D8FAFCA869F9F9AFD0DADE11
:10A58000FAD9F88F9FA8F1CCF398DB45D9AFDFD08B
:10A59000F8D8F18F9FA8CAF38809DAAF8FCBF8D823
:10A5A000F2AD978D0CD9A5DFF9BAA6F3FAF412F241
:10A5B000D8950DD1D9BAA6F3FADAA5F2C1BAA6F3A5
:10A5C000DFD8F1BAB2B68696A6D0CAF349DAA6CBDE
:10A5D000F8D8B0B4B8D8AD84F2C0DFF18FCBC3A83F
:10A5E000B2B68696C8C1CBC3F3B0B48898A821DBB5
:10A5F000718D9D71859521D9ADF2FAD88597A828DE
:10A60000D9F408D8F28D29DAF405D9F285A4C2F27A
:10A61000D8A88D9401D1D9F411F2D88721D8F40AA1
:10A62000D8F28498A8C801D1D9F411D8F3A4C8BB32
:10A63000AFD0F2DEF8F8F8F8F8F8F8F8D8F1B8F694
:10A64000B5B9B08A95A3DE3CA3D9F8D85CA3D9F8F4
:10A65000D87CA3D9F8D8F8F9D1A5D9DFDAFAD8B1DE
:10A660008530F7D9DED8F830ADDADED8F2B48C997F
:10A67000A32D557DA083DFDFDFB591A0F629D9FB9F
:10A68000D8A0FC29D9FAD8A0D051D9F8D8FC51D9F2
:10A69000F9D879D9FBD8A0D0FC79D9FAD8A1F9F9A1
:10A6A000F9F9F9A0DADFDFDFD8A1F8F8F8F8F8ACAB
:10A6B000DEF8ADDE8393AC2C547CF1A8DFDFDFF64F
:10A6C0009D2CDAA0DFD9FADB2DF8D8A850DAA0D07B
:10A6D000DED9D0F8F8F8DB55F8D8A878DAA0D0DFC2
:10A6E000D9D0FAF8F8F8F8DB7DF8D89CA88CF530CA
:10A6F000DB38D9D0DEDFA0D0DEDFD8A848DB58D9E0
:10A70000DFD0DEA0DFD0DED8A868DB70D9DFDFA025
:10A71000DFDFD8F1A888902C547C98A8D05C38D181
:10A72000DAF2AE8CDFF9D8B087A8C1C1B188A8C66B
:10A73000F9F9DA36D8A8F9DA36D8A8F9DA36D8A885
:10A74000F9DA36D8A8F9DA36D8F78D9DADF818DAE7
:10A75000F2AEDFD8F7ADFA30D9A4DEF9D8F2AEDE2A
:10A76000FAF983A7D9C3C5C7F1889BA77AADF7DEED
:10A77000DFA4F8849408A797F300AEF29819A48890
:10A78000C6A39488F632DFF28393DB09D9F2AADFFD
:10A79000D8D8AEF8F9D1DAF3A4DEA7F1889B7AD83D
:10A7A000F38494AE19F9DAAAF1DFD8A881C0C3C541
:10A7B000C7A39283F628ADDED9F8D8A350ADD9F857
:10A7C000D8A378ADD9F8D8F8F9D1A1DADEC3C5C7D6
:10A7D000D8A18194F818F2B089ACC3C5C7F1D8B834
:10A7E000B4B09786A8319B069907AB9728889BF051
:10A7F0000C201440B0B4B8F0A88A9A285078B79BBF
:10A80000A8295179247059446938644831F1BBABA7
:10A8100088002C547CF0B38BB8A804285078F1B091
:10A8200088B49726A85998BBABB38B02264666B06E
:10A83000B8F08A9CA82951798B2951798A247059BA
:10A840008B2058718A4469388B3940688A64483152
:10A850008B30496088F1AC002C547CF08CA8042823
:10A860005078F1889726A85998AC8C02264666F055
:10A87000899CA8295179247059446938644831A9C0
:10A880008809205970AB11384069A8193148608C8B
:10A89000A83C415C207C00F187981986A86E767EE2
:10A8A000A999882D557DD8B1B5B9A3DFDFDFAED02A
:10A8B000DFAAD0DEF2ABF8F9D9B087C4AAF1DFDFA6
:10A8C000BBAFDFDFB9D8B1F1A3978E60DFB084F200
:10A8D000C8F8F9D9DED89385F14AB183A308B583C6
:10A8E0009A0810B79F10D8F1B0BAAEB08AC2B2B60B
:10A8F0008E9EF1FBD9F41DD8F9D90CF1D8F8F8AD3A
:10A9000061D9AEFBD8F40CF1D8F8F8AD19D9AEFB8B
:10A91000DFD8F416F1D8F8AD8D61D9F4F4ACF59C1C
:10A920009C8DDF2BBAB6AEFAF8F40BD8F1AED0F8A6
:10A93000AD51DAAEFAF8F1D8B9B1B6A3839C08B933
:10A94000B1839AB5AAC0FD3083B79F10B58B93F23F
:10A950000202D1ABDADED8F1B080BAABC0C3B284A8
:10A96000C1C3D8B1B9F38BA391B609B4D9ABDEB0EA
:10A97000879CB9A3DDF1B38B8B8B8B8BB087A3A3A3
:10A98000A3A3B28BB69BF2A3A3A3A3A3A3A3A3A346
:10A99000A3F1B087B59AA3F39BA3A3DCBAACDFB94C
:10A9A000A3A3A3A3A3A3A3A3A3A3A3A3A3A3A3A377
:10A9B000D8D8D8BBB3B7F1AAF9DAFFD9809AAA28B8
:10A9C000B48098A720B79787A86688F07951F1904E
:10A9D0002C870CA781976293F0717160859401298F
:10A9E000517990A5F1284C6C870C95188578A38334
:10A9F00090284C6C886CD8F3A28200F210A89219AF
:10AA000080A2F2D926D8F188A84DD948D896A8397D
:10AA100080D93CD89580A839A68698D92CDA87A702
:10AA20002CD8A8899519A980D938D8A88939A9809E
:10AA3000DA3CD8A82EA83990D90CD8A8953198D945
:10AA40000CD8A809D9FFD801DAFFD89539A9DA2698
:10AA5000FFD890A80D8999A810809821DA2ED8895E
:10AA600099A83180DA2ED8A886963180DA2ED8A817
:10AA7000873180DA2ED8A88292F34180F1D92ED87E
:10AA8000A882F31980F1D92ED882ACF3C0A280221B
:10AA9000F1A62EA72EA92298A829DAACDEFFD8A20B
:10AAA000F22AF1A92E8292A8F23180A696F1D9005D
:10AAB000AC8C9C0C30ACDED0DEFFD88C9CACD010C3
:10AAC000ACDE8092A2F24C82A8F1CAF235F19688EF
:10AAD000A6D900D8F1FF00004FBB610567ACDD3F90
:10AAE000182D4454FB21E93F9BF681D20B73EF3FB5
:10AAF000182D4454FB21F93FE2652F227F2B7A3C2D
:10AB0000075C143326A6813CBDCBF07A8807703CE5
:10AB1000075C143326A6913CC4EB98999999C9BF58
:10AB2000711623FEC671BCBF6D9A74AFF2B0B3BF8D
:10AB30009AFDDE522DDEADBF2F6C6A2C44B4A2BF4D
:10AB40000D5555555555D53FFF8300922449C23FB9
:10AB50006E204CC5CD45B73F513DD0A0660DB13FED
:10AB6000EB0D76244B7BA93F11DA22E33AAD903FFF
:10AB7000000000000000000002400000000000A0F3
:10AB80000000000005400000000000C800000000B8
:10AB90000C4000000000409C000000001940000034
:10ABA0000020BCBE0000000034400000BFC91B8E66
:10ABB00000000004B5400000504BCFD06607E2CF44
:10ABC000010000006C4100003E8251AADFEEA73474
:10ABD00001000000D9420000DCB5A0E23A301F9726
:10ABE000FFFFFFFFB4450000FD25A0C8E9A3C14F4A
:10ABF000FFFFFFFFFF3F000000000080000000009B
:10AC0000FF3F0000000000800000000050726F64F1
:10AC1000756374204944207265616420617320303B
:10AC200020696E6469636174657320646576696325
:10AC3000652069732065697468657220696E636F49
:10AC40006D70617469626C65206F7220616E204D59
:10AC50005055333035302E0D0A00000098AC0008F6
:10AC600000000020200300006C010008B4AD0008C3
:10AC70002003002048070000C80100081C00000055
:10AC800043000000F8FFFFFF0C0000000E00000072
:10AC90000F0000002E0000001184A24A0468090180
:10ACA000020304060708090C6910051802040608C7
:10ACB00015404042CC000B1440A09E8282829EA090
:10ACC0002020000D113F908840432C1028464180E1
:10ACD000801C100C44012B45C606041144140C388A
:10ACE000098040201E2040407F2003124040380948
:10ACF00008884828180FE8080109111F2B080901C6
:10AD00003AFF0609112139C0080A1204F49494FF8D
:10AD10009494F404E1080D10201F20484442415F40
:10AD2000414244488029764C88780F7F0911601E83
:10AD30002010484641012A7F050911C029350B180A
:10AD4000C838402E08040201FF3C19010213FF0815
:10AD50000E12C8B88FE888C820900C030C902060B1
:10AD6000161808FF04041A3FC20414404070280952
:10AD7000FC242424FC252624080211040010114080
:10AD8000308F80844C55252525554C8080800009C6
:10AD90002C9A99193FCDCCCC3D024546C3803F5AF1
:10ADA000FF047201139C9E1B08900401209AB82492
:04ADB000693CC10039
:0400000508000131BD
:00000001FF
